:1000000051C1000077C1000075C1000073C100003C
:1000100071C100006FC100006DC100006BC1000024
:1000200069C1000067C1000065C1000063C1000034
:1000300061C100005FC100005DC100005BC1000044
:100040000C94502C57C100000C94651F53C1000044
:1000500051C100004FC100004DC100004BC1000064
:100060000C94B61247C1000000008207330FC71678
:10007000331EAD254F2D0A35D93CB6449C4C8554D2
:100080006C5C4A64196CD4737B7B0B83848AE49127
:100090002C995AA06FA765AE3CB5F0BB7EC2E7C8ED
:1000A0000000B200F9010F03E703A5043C05C405F5
:1000B0003806A306F9064907D10FAC0F680FFB0EEF
:1000C000580E770D550CFB0A810905089E0666053A
:1000D00061048303D4024602DA0183013F01070170
:1000E000DA00B6002000327DFF1F1F1F0000000055
:1000F0000000000000001F1F1F1F1F1F0000001F27
:100100001F0000000E0E0E0C080000000000001F73
:100110001F00000000030F0F1F000000001F1F1F23
:100120001F00000000181E1E1F1F0F0F03000000FD
:10013000001F1E1E18000000001F1F1F1F000000D0
:10014000000E0E0E0E0C0800000000000000001F44
:100150001F1C1C1C1E1E1F1F1F0707070F0F1F1F22
:100160001F1F1F1F1C1C1C1C1C181C1E0F07070711
:10017000071F1D1D1C1C1C1C1C1F1717070707072A
:10018000071C1C1C1C1C1F1F1F070707070F1E1C1A
:10019000181F0000000000001F1F00000E000000DC
:1001A0001F1F00040E0400001F1F0E1F1F1F1F0E25
:1001B0001F101010101010101018181818181818F8
:1001C000181C1C1C1C1C1C1C1C1E1E1E1E1E1E1E65
:1001D0001E000000000000001F0000000000001FC3
:1001E0001F00000000001F1F1F000000001F1F1F36
:1001F0001F0000001F1F1F1F1F00001F1F1F1F1FAA
:100200001F001F1F1F1F1F1F1F4253543A00503152
:100210003A004C42443A004147543A005448523A5A
:10022000004C4D4D3A2020202020204147543A00D8
:100230004C443A2020202020202052504D3A004D9E
:100240006178200000000000240027002A00000040
:100250000000250028002B000000000023002600DD
:100260002900040404040404040402020202020239
:10027000030303030303010204081020408001026A
:1002800004081020010204081020000000070002EA
:100290000100000304060000000000000000120E30
:1002A0003F11E72011241FBECFEFD8E0DEBFCDBF46
:1002B00013E0A0E0B1E0ECE6F5E702C005900D9296
:1002C000AC3BB107D9F715E0ACEBB3E001C01D9230
:1002D000A13BB107E1F712E0C4EAD2E004C02297E3
:1002E000FE010E945736CE39D107C9F70E941F0E72
:1002F0000C94B43A85CE08950895FC0120E030E0D6
:1003000040E050E080E6848B86EE858B80E090E0D4
:10031000A0E8BFE382839383A483B58381E0838BCA
:10032000268337834087518712861182108280E0AE
:1003300090E0A0ECB2E483879487A587B6872787EF
:10034000308B418B528B0895CF93DF93EC018B89D7
:10035000861709F43FC06B8B6130A1F480E090E018
:10036000A0E8BFE38A839B83AC83BD836F857889D4
:1003700089899A8920E030E040E050E00E94F9311C
:100380006C8913C080E090E0A0ECBFE38A839B837C
:10039000AC83BD836F85788989899A8920E030E0B4
:1003A00040E050E00E94F9316D89181654F470E075
:1003B00080E090E00E9425336F87788B898B9A8B41
:1003C00009C070E080E090E00E9425336B877C8755
:1003D0008D879E87DF91CF910895EF92FF920F93C3
:1003E0001F93CF93DF93EC0180911204909113043B
:1003F0000097E9F46F85788989899A8920E030E04F
:1004000040E050E00E94CE31882371F58B859C85B9
:10041000AD85BE858F87988BA98BBA8B80E090E0E5
:10042000A0E0B0E08B879C87AD87BE871DC0181603
:100430001906D4F4EF84F88809891A89C801B7012C
:1004400020E030E040E050E00E94F931181664F4FA
:10045000EB86FC860D871E8780E090E0A0E0B0E090
:100460008F87988BA98BBA8BDF91CF911F910F91BA
:10047000FF90EF900895FC018081813031F0813050
:1004800010F01082089581E001C082E08083089519
:10049000EF92FF920F931F93CF93DF93C0E0D0E0D2
:1004A000FE01EE0FFF1FE859FF4F059114916017F1
:1004B000710708F437C021969E01220F331F219740
:1004C000F901E859FF4F859194918617970750F1EC
:1004D000F901E859FF4FE590F490601B710B80E043
:1004E00090E022E330E040E050E00E948F35E01AD7
:1004F000F10A00E010E0A80197010E94EF3582E3C5
:1005000090E0C89FA001C99F500DD89F500D1124A5
:10051000420F531FCA01DF91CF911F910F91FF909E
:10052000EF9008952196CC31D10509F0B9CF40E084
:1005300050E0F0CFCF92DF92EF92FF920F931F9394
:10054000CF93DF9320E030E0F901EE0FFF1FE85476
:10055000FF4FC591D491C617D70708F445C069016C
:100560000894C11CD11C7601EE0CFF1CF701E85465
:10057000FF4F8591949168177907B0F1F701E8541E
:10058000FF4F05911491601B710B80E090E026EF06
:100590003FEF4FEF5FEF0E948F35C01BD10B9E01E5
:1005A00040E050E00E94EF35C60143E0880F991FFC
:1005B0004A95E1F78E0D9F1D820F931F4E9723E002
:1005C000883E920714F087EE93E02FEF883D920764
:1005D00014F488ED9FEFDF91CF911F910F91FF9061
:1005E000EF90DF90CF9008952F5F3F4F2631310578
:1005F00009F0AACF80E090E0E1CFCF92DF92EF92B6
:10060000FF920F931F93CF93DF93C0E0D0E06E0172
:10061000CC0CDD1CF601E056FF4F059114916017DC
:10062000710708F442C021969E01220F331F2197C3
:10063000F901E056FF4F8591949186179707A8F12D
:10064000F901E056FF4FE590F490601B710B80E0DC
:1006500090E02AE030E040E050E00E948F35E01A60
:10066000F10A00E010E0A80197010E94EF35CE01E9
:10067000B3E0880F991FBA95E1F78C0D9D1D820F8D
:10068000931F0A9723E0883E920714F087EE93E0C9
:1006900097FF02C080E090E0DF91CF911F910F9112
:1006A000FF90EF90DF90CF9008952196CC30D10548
:1006B00009F0ADCF80E090E0E4CF70E0FB01F89668
:1006C0002CEB33E0EE0FFF1FE20FF31F8091EA03E4
:1006D0009091EB0391838083FB017E96EE0FFF1FC9
:1006E000EE0FFF1FE20FF31F8091FE039091FF03B7
:1006F000A0910004B091010480839183A283B3830D
:10070000FB01B296EE0FFF1FEE0FFF1FE20FF31F6C
:100710008091100490911104AA2797FDA095BA2FFB
:1007200080839183A283B3836A5D7F4FFB01EE0FC9
:10073000FF1FEE0FFF1FE20FF31F8091180490912F
:100740001904A0911A04B0911B0480839183A283A1
:10075000B383625D7F4F660F771F260F371F80912F
:10076000220490912304F90191838083089580915C
:100770007004823001F1833020F4813009F041C0EF
:1007800005C0873021F18830E1F532C080E090E08B
:10079000A0E0B0E08093E2039093E303A093E4032E
:1007A000B093E5038091E8039091E9039093E70308
:1007B0008093E60308958CE694E00E94E71988EEA2
:1007C00094E069E670E0409171040C94F70E8CE6B9
:1007D00094E066E00E946B14FC01009791F0128691
:1007E000118688E893E194878387CF010C948D1D4F
:1007F0008CE694E067E00E946B14009711F00C9473
:100800008A1E089520917004223029F0233049F087
:10081000213041F430CE80917004909171040C9499
:10082000FE1B29CE08950F931F938C018CE694E054
:100830000E94841B0E94982C605F784D8F4F9F4FC1
:10084000F80164837583868397831F910F910895C0
:100850002091100430911104C90180579741855FA0
:10086000914020F483E068E270E007C089E124361B
:1008700038072CF083E06FEF70E00C945A2D20576E
:1008800037412CF483E060E070E00C945A2D089519
:10089000DF92EF92FF920F931F93CF93DF93EC01C0
:1008A000D09071042091EA033091EB038091EC0326
:1008B0009091ED03815B94401CF4215B344054F033
:1008C0000E94982C68577C4E8F4F9F4F6E877F8772
:1008D000888B998BEE84FF84088919890E94982C53
:1008E000E616F70608071907E0F0EA88FB880C8986
:1008F0001D890E94982C6E157F0580079107E8F0EE
:10090000DD2019F492E0D92E01C0DD240E94982C3C
:100910006C597F4F8F4F9F4F6A8B7B8B8C8B9D8B3E
:1009200007C088EE94E069E670E00E94FB0ED82EC6
:100930008CE694E06D2D0E94D9198CE694E06D2D23
:100940000E94D919DF91CF911F910F91FF90EF90E5
:10095000DF900895AF92BF92CF92DF92EF92FF9215
:100960000F931F938091020490910304A0910404BB
:10097000B09105048093DE039093DF03A093E0031E
:10098000B093E10300D000D06091BE037091BF032B
:10099000882777FD8095982F28EC30E040E050E0E4
:1009A000EDB7FEB7218332834383548320E030E0E8
:1009B00040E050E0E12CE0E1FE2E012D112DAA24B3
:1009C000BB2465010E94EC232AE030E040E050E0C7
:1009D0000E94EF353093E9032093E8030F900F90C6
:1009E0000F900F9088EE94E06DEC70E0422F0E9423
:1009F000F70E6091DE037091DF038091E003909128
:100A0000E10320E030E04AE754E40E9432300E94E3
:100A1000D432AB01BC0188EC90E00E94BA0E80E0B9
:100A200090E0A0E0B0E08093E2039093E303A09312
:100A3000E403B093E5038091E8039091E903909378
:100A4000E7038093E60300E915E0C80160E071E088
:100A50000E94F122C80162E071E00E945821409199
:100A6000DE035091DF036091E0037091E103C80160
:100A700022E030E00E94E3231F910F91FF90EF905E
:100A8000DF90CF90BF90AF9008959C01809170044B
:100A9000813011F4C9015ECF0895CF93DF93EC014B
:100AA000605870406230710529F16330710509F4B6
:100AB00044C06130710509F044C08AA99BA9ACA962
:100AC000BDA90097A105B10519F4CE019BDE2EC08A
:100AD0000E94982C2AA93BA94CA95DA928513C4FFA
:100AE0004F4F5F4F621773078407950750F1CE0190
:100AF0009ADE1CC08AA99BA9ACA9BDA90097A10533
:100B0000B10519F4CE0133DE11C00E94982C2AA938
:100B10003BA94CA95DA928513C4F4F4F5F4F62172D
:100B200073078407950768F0CE01AFDF0E94982C09
:100B30006AAB7BAB8CAB9DAB04C01AAA1BAA1CAAE8
:100B40001DAADF91CF9108950F931F93DF93CF9349
:100B500000D0CDB7DEB78C01FC018081833009F471
:100B60005EC080E995E06DE071E00E94582180E967
:100B700095E06FE071E00E9458214091D4045091BB
:100B8000D5046091D6047091D70480E995E022E005
:100B900030E00E94E22380E995E060E071E00E948D
:100BA00058214091FE035091FF0360910004709121
:100BB000010480E995E022E030E00E94E22380E930
:100BC00095E060E071E00E9458214091DD04509171
:100BD000DE046091DF047091E00480E995E022E09A
:100BE00030E00E94E22380E995E060E071E00E943D
:100BF00058218091D2049091D304892B31F480E95B
:100C000095E064E171E00E94582180E995E06DE192
:100C100071E00E94582180E995E00E94A42280E9B9
:100C200095E06DE071E00E945821F80180818130EB
:100C300049F0813008F499C1823079F1833009F0AC
:100C400092C149C1F801408551856285738580E96B
:100C500095E02AE030E00E941F2280E995E06FE1F4
:100C600071E00E9458210EEB13E0F801619171913F
:100C70008F0180E995E04AE050E00E94812280E9FE
:100C800095E06FE171E00E945821F3E00C3D1F07F1
:100C900061F7F8016081718117C180E995E062E038
:100CA00070E04AE050E00E94812280E995E061E234
:100CB00071E00E945821F801408551856285738555
:100CC00080E995E02AE030E00E941F2280E995E06B
:100CD0006FE171E00E94582160911004709111043D
:100CE00080E995E04AE050E00E94812280E995E0A9
:100CF0006FE171E00E9458214091FE035091FF0383
:100D0000609100047091010480E995E022E030E0F8
:100D10000E94E22380E995E06FE171E00E94582192
:100D2000609112047091130480E995E04AE050E06C
:100D30000E94812280E995E06FE171E00E945821D4
:100D400040910604509107046091080470910904D1
:100D500080E995E022E030E00E94E22380E995E01E
:100D60006FE171E00E9458214091180450911904DC
:100D700060911A0470911B0480E995E022E030E054
:100D80000E94E22380E995E06FE171E00E94582122
:100D90004091140450911504609116047091170449
:100DA00080E995E022E030E00E94E22380E995E0CE
:100DB0006FE171E00E9458216091EA037091EB03AA
:100DC00080E995E04AE050E00E94812280E995E0C8
:100DD0006FE171E00E9458216091EC037091ED0386
:100DE00080E995E04AE050E00E94812280E995E0A8
:100DF0006FE171E00E94582140912804509129042C
:100E000060912A0470912B0480E995E022E030E0A3
:100E10000E94E22380E995E06FE171E00E94582191
:100E2000609122047091230480E995E04AE050E04B
:100E30000E94812280E995E06FE171E00E945821D3
:100E4000609124047091250480E995E04AE050E027
:100E50000E94812280E995E06FE171E00E945821B3
:100E6000609126047091270480E995E04AE050E003
:100E70000E94812280E995E06FE171E00E94582193
:100E800060911C0470911D0480E995E04AE050E0F7
:100E90000E94812280E995E06FE171E00E94582173
:100EA00060911E0470911F0480E995E04AE050E0D3
:100EB0000E94812280E995E06FE171E00E94582153
:100EC000609120047091210480E995E04AE050E0AF
:100ED0000E9481224AC080E995E060E174E042E02E
:100EE00050E00E94392180E995E062E174E042E03F
:100EF00050E00E94392160910604709107048091AE
:100F0000080490910904D4D69A8389838E010F5FD7
:100F10001F4F80E995E0B80142E050E00E9439217E
:100F2000609102047091030480910404909105047F
:100F3000BFD69A83898380E995E0B80142E050E00A
:100F40000E94392180E995E06AEE73E042E050E0CA
:100F50000E94392180E995E06CEE73E042E050E0B8
:100F60000E94392102C0F801108280E995E06DE10C
:100F700071E00E94582180E995E00E94A42273D676
:100F8000BC0180E995E04AE050E00E94C2220F9047
:100F90000F90CF91DF911F910F910895EF92FF92E3
:100FA0000F931F9388EE94E069E670E024D7682FD2
:100FB0008CE694E00E94D91988EE94E06DEC70E024
:100FC0001AD7853128F490E09093E9038093E803E1
:100FD00088EC90E086D60E947A3220E030E04AE742
:100FE00054E40E9427317B018C0120E030E040E096
:100FF00050E00E94F931181694F4C801B7012AE9AB
:1010000039E949E95FE30E944F32882344F4E092D2
:10101000DE03F092DF030093E0031093E1031F91DE
:101020000F91FF90EF900895DF92EF92FF920F9350
:101030001F93CF93DF938C017C01C0E0D0E0DD24CF
:10104000DA9410C080E995E00E94A420D82E06C052
:1010500080E995E00E94A420F701818F21960894F1
:10106000E11CF11C80E995E00E947920892B31F088
:10107000C931D10531F0209729F3EACFC931D10523
:1010800089F5F1E0FD1570F1F801628D738D848DA5
:10109000958D0E947A3220E030E04AE754E40E94C5
:1010A00027316093D4047093D5048093D604909331
:1010B000D704DD2009F05AC0F80162A173A184A110
:1010C00095A10E947A3220E030E04AE754E40E9481
:1010D00027316093DD047093DE048093DF049093E6
:1010E000E00444C0F3E0DF1619F184E0D81671F192
:1010F000E2E0DE1609F03AC02297C4F1F801828DD1
:10110000823069F0833018F4813081F505C0833076
:1011100049F0843059F509C0C80174DB27C0C80103
:1011200082DB24C0C80123DB21C0C801AEDC1EC0A5
:101130002297E4F0F801828D823029F08330B1F4F7
:10114000F801D08213C0F801808310C0C230D105ED
:101150006CF0F801828D843049F424973CF0F8015A
:10116000838D8093E604848D8093E70480E995E085
:101170000E94C820DF91CF911F910F91FF90EF90B7
:10118000DF900895CF93DF93EC012D96CE0160E2BE
:1011900070E041E050E00E94B011CE010E94E610E4
:1011A000882319F0CE010E94EC10DF91CF910895B1
:1011B000CF93DF93EC012D96CE0161E270E041E028
:1011C00050E00E94B011CE010E94E610882319F071
:1011D000CE010E94EC10DF91CF910895FF920F9302
:1011E0001F93F62E8C01035F1F4FC80160E270E071
:1011F000ECD7C8016F2D0E944011C8010E949111C7
:101200001F910F91FF900895FF920F931F93F62E59
:101210008C01035F1F4FC80161E270E0D6D7C8019F
:101220006F2D0E944011C8010E9491111F910F91D2
:10123000FF900895CF92DF92EF92FF920F931F934A
:10124000CF93DF938C01D62EFC018485F8E0F6174E
:1012500030F48D77F8018487862F885004C08E770C
:10126000F8018487862F90E00197B3E0880F991FDB
:10127000BA95E1F7A0ECCA2EC82AC801F801648526
:10128000ADDFC7E0D0E0F1E0EF2EF12CC7010C2E6E
:1012900002C0880F991F0A94E2F76C2D682381E140
:1012A0000E940B2E8DE061E00E940B2E8DE060E02D
:1012B0000E940B2E2197C230D10541F78DE061E0ED
:1012C0000E940B2E8DE060E00E940B2E8DE061E00D
:1012D0000E940B2E8DE060E00E940B2EEE24FF2476
:1012E000CBE0D0E08CE00E943F2E0C2E02C0880F95
:1012F000991F0A94E2F7E80EF91E8DE061E00E9462
:101300000B2E8DE060E00E940B2E2197FFEFCF3F68
:10131000DF0741F7F8018485F8E0FD1510F48268D5
:1013200001C08168F8018487C801F801648556DF2F
:10133000C701DF91CF911F910F91FF90EF90DF9048
:10134000CF900895AF92BF92CF92DF92EF92FF922B
:101350000F931F93DF93CF93CDB7DEB760970FB690
:10136000F894DEBF0FBECDBF7C01DE011196E5E330
:10137000F1E080E101900D928150E1F7CC24DD2471
:101380005E010894A11CB11CF501EC0DFD1D8081CE
:101390009181880F991F880F991FF7016485637EDB
:1013A000682B6487C7011ADF64E170E080E090E099
:1013B0000E94CC2CC70160E13DDFAA2797FDA095D4
:1013C000BA2FBC01CD010E947A3220E030E040EA21
:1013D00050E40E94323020E030E040E859E30E94BF
:1013E000323020E030E44CE156E40E9432300E947A
:1013F0006E2E9B01AC01C701B9014AD88C01F4E003
:1014000082399F0718F060E070E00CC0609114040E
:101410007091150480911604909117040E94D432A3
:10142000600F711FF601E454FC4F77A766A7809107
:101430003204909133046817790718F0C70163E00C
:101440003CD982E090E0C80ED91E94E0C916D104C0
:1014500009F09ACF60960FB6F894DEBF0FBECDBFED
:10146000CF91DF911F910F91FF90EF90DF90CF9080
:10147000BF90AF900895AF92BF92CF92DF92EF925C
:10148000FF920F931F93CF93DF93EC016091BE0304
:101490007091BF03882777FD8095982F0E947A323C
:1014A00020E030E040EA50E40E94323020E030E0BA
:1014B00040E859E30E94323020E030E040E151E45E
:1014C0000E94323020E030E040E751E40E94E02FFB
:1014D00021E73FE048E651E40E9427317B018C017F
:1014E0006093FE037093FF038093000490930104C4
:1014F0002091DE033091DF034091E0035091E1033E
:101500000E940B30609302047093030480930404E0
:1015100090930504C801B701209138043091390433
:1015200040913A0450913B040E94243288231CF0DD
:10153000CE0161E0C2D8E090D203F090D30300273F
:10154000F7FC0095102FC801B7010E947A3220E005
:1015500030E040E859E30E94323020E030E040EAD9
:1015600050E40E9432309B01AC010E940B3020E01D
:1015700030E040E251E40E940B3060930A04709323
:101580000B0480930C0490930D0423E333E34BE6A8
:1015900051E40E94273160930604709307048093FE
:1015A00008049093090400D000D088EC90E0A0E0FB
:1015B000B0E0EDB7FEB781839283A383B483C80103
:1015C000B70120E030E040E050E0E12CF0E1FF2EF8
:1015D000012D112DAA24BB2465010E94EC230F903C
:1015E0000F900F900F90693C710514F068EC70E05B
:1015F00077FF02C060E070E070930F0460930E0408
:101600006091140470911504809116049091170450
:1016100026E636E646E65FE30E9432307B018C0127
:101620006091DA037091DB03882777FD8095982F0E
:101630000E947A3220E030E04AEF53E40E943230D8
:1016400020E030E040E859E30E9432302DEC3CECE1
:101650004CEC5DE30E9432309B01AC01C801B70144
:101660000E940B3060931404709315048093160449
:101670009093170400D000D06091D4037091D503EB
:10168000882777FD8095982F24E630E040E050E0F1
:10169000EDB7FEB721833283438354832CE632E0D7
:1016A00040E050E0EAECEE2EEDE0FE2E012D112D93
:1016B000AA24BB2465010E94EC230F900F900F9089
:1016C0000F906536710514F064E670E077FF02C094
:1016D00060E070E084E690E0861B970B9093130423
:1016E000809312046091D8037091D903882777FD05
:1016F0008095982F0E947A3220E030E040EA50E452
:101700000E94323020E030E040E859E30E9432305D
:10171000609318047093190480931A0490931B0427
:101720006091FA037091FB032091F8033091F90363
:10173000F901EE0FFF1FE251FC4F40815181809172
:10174000D6039091D70391838083680F791F641B20
:10175000750B7093FB036093FA032F5F3F4F309339
:10176000F9032093F8032530310524F01092F90392
:101770001092F803CB0165E070E00E94BA357093D7
:10178000FD036093FC03882777FD8095982F0E94C6
:101790007A322FE832EC45E150E40E9432300E9468
:1017A000D4327093110460931004882777FD8095DC
:1017B000982F20914C0430914D0440914E0450914B
:1017C0004F04621773078407950724F0CE0162E087
:1017D0000E945D0380E00E94382DAA2797FDA09506
:1017E000BA2FBC01CD010E947A3220E030E040EAFD
:1017F00050E40E94323020E030EC4FE754E40E9485
:10180000273128E431EE42E850E40E94323023E3ED
:1018100033E343E35FE30E940B306093280470934B
:10182000290480932A0490932B048A81813011F437
:10183000CE0188DD6091C2037091C303CE010E9486
:101840009A0290931D0480931C046091C4037091CC
:10185000C503CE010E949A0290931F0480931E0438
:101860006091C6037091C703CE010E949A029093C3
:101870002104809320046091C8037091C903CE01B4
:101880000E94FD0290932304809322046091CA0376
:101890007091CB03CE010E94FD02909325048093AA
:1018A00024046091CC037091CD03CE010E94FD020F
:1018B0009093270480932604DF91CF911F910F917D
:1018C000FF90EF90DF90CF90BF90AF900895EF9290
:1018D000FF921F93CF93DF93EC010E94982C6887AF
:1018E00079878A879B87AEEBEA2EA3E0FA2E11E078
:1018F000CE01612F9FDCF701819391937F011F5FE0
:101900001131B1F7CE01B7DDCE010E9428048CE67B
:1019100094E00E946A1BCE014BDC682F70E0CE0180
:10192000BCD80E94982C2C813D814E815F8162172A
:1019300073078407950778F088EE94E064E670E01A
:101940004091700454D280EC9FE1A8E9B9E18C8306
:101950009D83AE83BF838FE00E943F2EBC0182ED4A
:1019600094E00E94A40182ED94E00E94ED01609158
:10197000DD047091DE048091DF049091E0040E9408
:10198000D4329B01AC018BE0B9010E945A2D0E9418
:10199000982C2E893F89488D598D2617370748077F
:1019A000590778F4CE0140DBCE01CED88E899F89CD
:1019B000A88DB98D4496A11DB11D8E8B9F8BA88FCC
:1019C000B98FDF91CF911F91FF90EF9008950D9601
:1019D000F1C30D96EFC3EF92FF920F931F93DF9326
:1019E000CF930F92CDB7DEB77C018FEFF7018487DD
:1019F000CE010196DFD3F70116861786108A118A69
:101A0000128A138A148A158A148215821682178202
:101A1000108611861286138680E090E0A0E0B0E088
:101A20008093E2039093E303A093E403B093E50370
:101A30001092E7031092E60381E08383808312AA69
:101A400013AA14AA15AA85E061E00E94B82D8FE0C0
:101A500060E00E94B82D8FE061E00E940B2E8BE0C9
:101A600061E00E94B82DE1EBF0E080818760808327
:101A700081E161E00E94B82D8CE060E00E94B82D09
:101A80008DE061E00E94B82D81E160E00E940B2EA4
:101A90008DE060E00E940B2E00E915E0C80140E0F7
:101AA00051EE60E070E00E94F61FC7010D9659D418
:101AB000C701F701648592DBC80163E271E00E940F
:101AC000F122C7016BDA0CE614E0C80160ED77E0A3
:101AD0000E94F219C8010E94771BC70163E894DBDA
:101AE0000E94982CF701668B778B808F918F0F90D7
:101AF000CF91DF911F910F91FF90EF90089508957E
:101B00000895CF93DF93EC0180E090E0FE01E80FB1
:101B1000F91F11821082029682329105B9F780E096
:101B200090E0A0E8BFE38AA39BA3ACA3BDA380E0A1
:101B300090E0A0E0B0E08EA39FA3A8A7B9A71BA642
:101B40001AA61DA61CA61DAE1CAE1FAE1EAEC05C06
:101B5000DF4F1992199289939993A993B993888326
:101B60009983AA83BB832C9619821882289789931C
:101B70009993A993B99388839983AA83BB83269663
:101B8000199219921992199289939993A993B993D9
:101B900089939993A993B9931992199219921992C9
:101BA00019921992199219921992199219921992DD
:101BB00088839983AA83BB83CC56D040DE01A05989
:101BC000BF4FFE01E858FF4F80E090E020E030E09A
:101BD00040E050E011961C921E9220833183428394
:101BE0005383108A118A128A138A20A331A342A335
:101BF00053A3D9961C921E92D897019612963496AA
:101C00008430910539F71BAA1AAA1DAA1CAA1FAA7B
:101C10001EAA19AE18AE1BAE1AAE1FA61EA6DF91E5
:101C2000CF9108958CEB93E06BDF8CE694E052D675
:101C30008CE994E0CCDE82ED94E00C947C010E946F
:101C4000FA2C8CEB93E05DDF8CE694E00E948E1B17
:101C50008CE994E0C0DE82ED94E00E947D018CE985
:101C600094E035DEFCCF4091AD055091AE054115B5
:101C7000510521F44091B3035091B4032091B50371
:101C80003091B6032115310549F48DB7282F30E086
:101C90008091B1039091B203281B390B421753076F
:101CA00018F080E090E00895C901841B950B089519
:101CB00020E030E048EC52E40E9432300E94D432FE
:101CC000DC01CB010895AA2797FDA095BA2FBC018E
:101CD000CD010E947A3220E030E048EC52E40C94CE
:101CE00027318F929F92AF92BF92CF92DF92EF9265
:101CF000FF920F931F936C0158EEA52E54E0B52E62
:101D0000C501B60178D0882E0894C11CD11CC5012C
:101D1000B60171D0E82E0894C11CD11CC501B601D2
:101D20006AD0982E0894C11CD11CC501B60163D09D
:101D300090E0982F8827890D911DA0E0B0E0DC018C
:101D400099278827FF24FE2CEE24E80CF11C00E0E4
:101D500010E08E0D9F1DA01FB11FBC01CD011F9172
:101D60000F91FF90EF90DF90CF90BF90AF909F903A
:101D70008F900895AF92BF92CF92DF92EF92FF9231
:101D80000F931F938C016A017B01F8EEAF2EF4E0F4
:101D9000BF2EC501B8014C2D2AD00F5F1F4F55270C
:101DA000F7FC5A954F2D3E2D2D2DC501B801422F20
:101DB0001ED00F5F1F4F9701552737FD5095452FB8
:101DC000C501B801422F13D00F5F1F4FCF2CDD2468
:101DD000EE24FF24C501B8014C2D09D01F910F91AD
:101DE000FF90EF90DF90CF90BF90AF900895CB0120
:101DF000642F0C94933ACB010C948B3A709354015A
:101E000060935301615070406230710530F081E0A1
:101E100090E090935401809353010895709354017E
:101E200060935301615070406230710530F081E081
:101E300090E090935401809353010895809149015B
:101E400060E00E940B2E00008091490161E00E9439
:101E50000B2E00008091490160E00E940B2E0000D3
:101E60000895EF92FF920F931F93CF93DF937C011E
:101E70008B010F701070C0914B01D0914C0108C0C4
:101E8000602F61708C2F0E940B2E1595079521965F
:101E900080915101909152018C179D078CF7C701D9
:101EA000CDDFDF91CF911F910F91FF90EF900895BB
:101EB000EF92FF920F931F938C017B0194E0759535
:101EC00067959A95E1F7C801CCDF8FE0E822FF24FF
:101ED000C801B701C6DF1F910F91FF90EF900895E1
:101EE0000F931F93CF93DF93EC018B0180914501FA
:101EF00060E00E940B2E8091E9049091EA04892B06
:101F000029F08091470160E00E940B2ECE01B801BC
:101F1000A8DFDF91CF911F910F9108951F93CF9369
:101F2000DF93EC01162F8091450161E00E940B2E9A
:101F30008091E9049091EA04892B29F0809147016E
:101F400060E00E940B2EE12FF0E0E4916E2F70E034
:101F5000CE01AEDFDF91CF911F910895EF92FF92F6
:101F60000F931F93CF93DF937C01042FEB0110E0BD
:101F700004C0C7016991D2DF1F5F1017D0F3DF9152
:101F8000CF911F910F91FF90EF9008950F931F93A2
:101F9000CF93DF93EC018B018091450161E00E94BA
:101FA0000B2E8091E9049091EA04892B29F080910D
:101FB000470160E00E940B2ECE01B80179DFDF916E
:101FC000CF911F910F9108950F931F93CF93DF939C
:101FD0008C01EB0106C02196F901649170E0C80103
:101FE000D5DF9E01FE0184918823A9F7DF91CF916F
:101FF0001F910F91089564EE70E0E6CFEF92FF928B
:102000001F93CF93DF937C01EB0110E007C0AC0F6F
:10201000BD1F6C9170E0C701B9DF1F5FA12FB0E059
:10202000FE0101900020E9F73197EC1BFD0BAE1784
:10203000BF0768F3DF91CF911F91FF90EF90089554
:10204000FB01E4916E2F70E0A1CF0F931F93CF930C
:10205000DF93EC018B018091450160E00E940B2E23
:102060008091E9049091EA04892B29F0809147013D
:1020700060E00E940B2ECE01B8011ADFDF91CF91F4
:102080001F910F910895EF92FF920F931F938C0170
:102090007A0170E0DADFC801B70196DF1F910F9176
:1020A000FF90EF900895CF93DF93EC018091490169
:1020B00061E00E94B82D8091450161E00E94B82D39
:1020C0008091E9049091EA04892B29F080914701DD
:1020D00061E00E94B82D80914B0161E00E94B82D13
:1020E00080914D0161E00E94B82D80914F0161E027
:1020F0000E94B82D8091510161E00E94B82D62E3E9
:1021000070E080E090E00E94CC2CCE0163E070E0B3
:10211000E7DE65E070E080E090E00E94CC2CCE012C
:1021200063E070E0DDDE84E690E00E94F02CCE01FA
:1021300063E070E0D5DE65E070E080E090E00E9452
:10214000CC2CCE0162E070E0CBDECE0162E070E02C
:10215000C7DECE0168E070E0C3DE8CE390E00E9451
:10216000F02CCE016CE070E070DF8CE390E00E9418
:10217000F02CCE0161E070E068DF63E070E080E0A9
:1021800090E00E94CC2CCE0166E070E05EDF61E062
:1021900070E080E090E00E94CC2CDF91CF91089518
:1021A00061E070E052DF61E070E080E090E00C946C
:1021B000CC2C0895089581E08093F4046093EF049B
:1021C0001092F2041092F3040895F5CF8091EE047A
:1021D0009091ED04891B08959091ED048091EE0497
:1021E000981710F080E00895E091EB04F091EC0472
:1021F000E90FF11D80819F5F9093ED0408959C018C
:102200008091F7049091F804892B11F19091ED04DD
:102210008091EE049817E0F090E00BC0E091EB04A1
:10222000F091EC04EA0FFB1FA20FB31F8C91808387
:102230009F5FA92FB0E0A617B70784F31092ED04B3
:102240006093EE04E091F704F091F804CB01099556
:102250000895E091F504F091F604309729F010927A
:10226000F2041092F304099508957093F8046093B2
:10227000F70408957093F6046093F50408950895A3
:10228000DF93CF930F92CDB7DEB769838091F404CB
:102290008823A9F08091F3048032A8F48091F2049D
:1022A000E091F004F091F104E80FF11D608380915A
:1022B000F2048F5F8093F2048093F30404C0CE0194
:1022C000019661E014D10F90CF91DF910895D8CF9E
:1022D000EF92FF920F931F93CF93DF937C01042F14
:1022E0008091F404882351F0EB0110E004C0C70191
:1022F0006991C6DF1F5F1017D0F303C0CB01642FB5
:10230000F6D0DF91CF911F910F91FF90EF9008953C
:10231000FB0101900020E9F73197E61BF70B4E2FE8
:10232000D7CF6091F0047091F1048091EF04409157
:10233000F30421E097D01092F2041092F30410926B
:10234000F4040895862F6091EB047091EC044132FF
:1023500008F040E24FD01092ED048093EE0408950F
:10236000F1CF80E290E061E070E00E94EA36909365
:10237000EC048093EB041092ED041092EE0480E2E2
:1023800090E061E070E00E94EA369093F10480935F
:10239000F0041092F2041092F3046AC20F931F9398
:1023A0008C01862F23D089E291E1C3D08FEF90E199
:1023B000BBD0C801D6DF1F910F910895EFCFFC016C
:1023C00020E030E08081882311F421E030E0C90171
:1023D0000895FC0181E08083089508950895009791
:1023E00011F00C94B13708950C940437880F809342
:1023F000BA000895982F413210F040E031C080912A
:10240000FA048823E1F781E08093FA048FEF809348
:102410000B05109202054150409303054F5F990F41
:1024200091609093FB0485EE8093BC008091FA0448
:102430008130E1F380910205841710F44091020588
:10244000A0910005B091010520E030E007C0FB013C
:10245000E20FF31F8D9180832F5F3F4F2417B8F356
:10246000842F08951F93582F122F413210F081E0CE
:102470003CC08091FA048823E1F782E08093FA045B
:102480008FEF80930B051092020540930305A091F6
:102490000005B0910105FB0102C081918D938E2F43
:1024A000861B8417D0F3852F90E0880F991F8093A7
:1024B000FB0485EE8093BC00112321F08091FA0487
:1024C0008230E1F380910B058F3F11F480E00DC065
:1024D00080910B05803211F482E007C080910B05DA
:1024E000803311F084E001C083E01F910895482FEC
:1024F000613210F081E008958091FA04843011F087
:1025000082E0089560930705A0910405B091050548
:10251000842F9C01F90102C081918D938E2F841B21
:102520008617D0F380E008959093FF048093FE0413
:1025300008959093FD048093FC040895882311F07E
:1025400085EC01C085E88093BC00089585ED8093FB
:10255000BC008091BC0084FDFCCF1092FA04089569
:1025600085EC8093BC001092FA0408951F920F929C
:102570000FB60F9211242F933F934F935F936F9356
:102580007F938F939F93AF93BF93EF93FF9380912C
:10259000B90090E0887F90708036910509F4E2C020
:1025A00081369105CCF58832910509F47BC08932DA
:1025B0009105B4F48031910509F46FC08131910522
:1025C0003CF4009709F438C1089709F040C165C090
:1025D0008831910509F466C0809709F038C17FC041
:1025E0008034910509F4A3C08134910544F480330B
:1025F000910509F47FC0C89709F029C186C08035CC
:10260000910509F486C08835910509F495C0883490
:10261000910509F01CC19EC08839910509F404C1D7
:1026200089399105ECF48837910509F49BC0893705
:1026300091054CF48836910509F494C080379105D2
:1026400009F005C18FC08838910509F4EDC08039C3
:10265000910509F48DC08038910509F0F8C088C053
:10266000803B910509F4B2C0813B91054CF4803A5E
:10267000910509F491C0883A910509F0E8C0A6C017
:10268000803C910509F4D4C0883C910509F4D0C080
:10269000883B910509F0DBC0B1C08091FB048093B9
:1026A000BB00C0C09091020580910305981778F493
:1026B00090910205E0910005F0910105E90FF11DEF
:1026C00080818093BB009F5F90930205ABC085ED36
:1026D0008093BC008091BC0084FDFCCFB6C080E23A
:1026E00080930B0585ED8093BC008091BC0084FD38
:1026F000FCCFABC080E380930B0585ED8093BC00DD
:102700008091BC0084FDFCCFA0C088E380930B05C2
:102710008FC0809102059091BB00E0910005F0917F
:102720000105E80FF11D90838F5F80930205909162
:1027300002058091030574C0809102059091BB0051
:10274000E0910005F0910105E80FF11D90838F5F86
:102750008093020585ED8093BC008091BC0084FDD0
:10276000FCCF73C083E08093FA0410920A055AC02C
:1027700080910A05803208F057C080910A05909137
:10278000BB00E0910805F0910905E80FF11D908369
:102790008F5F80930A0546C080910A05803248F415
:1027A00080910A05E0910805F0910905E80FF11DF7
:1027B000108260910A05E091FE04F091FF0480917F
:1027C00008059091090570E0099532C084E0809376
:1027D000FA041092060510920705E091FC04F091AE
:1027E000FD04099580910705882341F481E08093D9
:1027F0000705E0910405F09105051082909106050A
:10280000E0910405F0910505E90FF11D80818093A9
:10281000BB009F5F90930605909106058091070588
:10282000981710F485EC01C085E88093BC000FC0B8
:1028300085EC8093BC0009C010920B0585ED809358
:10284000BC008091BC0084FDFCCF1092FA04FF9183
:10285000EF91BF91AF919F918F917F916F915F9118
:102860004F913F912F910F900FBE0F901F90189591
:102870001092FA04449A459AE9EBF0E080818E7F49
:10288000808380818D7F808388E48093B80085E495
:102890008093BC0080E290E061E070E00E94EA3644
:1028A000809300059093010580E290E061E070E084
:1028B0000E94EA36809304059093050580E290E03B
:1028C00061E070E00E94EA36809308059093090564
:1028D000089508950895623018F080E090E008951A
:1028E000E62FF0E03196EE0FFF1FE80FF91F808111
:1028F00091810895FC01662309F4148208950F93D1
:102900001F93CF93DF93EC018A0167FF04C070E04F
:10291000888199819ADB88819981B8016FDBDF9189
:10292000CF911F910F910895FF920F931F93CF9313
:10293000DF93EC01262F277019F43EEFF32E01C030
:10294000F22E862F90E0821B910968E070E00E94D1
:10295000BA35623009F460C0633030F4662359F050
:10296000613009F0ACC035C0633009F46DC064302B
:1029700009F0A5C076C0042F10E000581F4F8881D1
:102980009981B80162DB888199816EEF70E0FEDA8F
:10299000005C1F4F88819981B80157DB888199813C
:1029A0006EEF70E0F3DA0C52104088819981B80123
:1029B0004CDB888199816EEF70E0E8DA005C1F4F94
:1029C00088819981B80141DB6F2D70E08881998100
:1029D00075C0042F10E000581F4F88819981B801FD
:1029E00034DB888199816EEF70E0D0DA005C1F4F94
:1029F00088819981B80129DB888199816EEF70E027
:102A0000C5DA0C52104088819981B8011EDB6F2D08
:102A100070E08881998147C0042F10E000581F4F53
:102A200088819981B80111DB888199816EEF70E00E
:102A3000ADDA005C1F4F88819981B80106DB6F2DEC
:102A400070E08881998124C0042F10E000581F4F46
:102A500088819981B801F9DA6F2D70E088819981B8
:102A60000CC0042F10E000581F4F88819981B801D5
:102A7000ECDA888199816FEF70E088DA005C1F4F93
:102A800088819981B801E1DA888199816FEF70E0DE
:102A90007DDA0C52104088819981B801D6DA88819C
:102AA00099816FEF70E072DA005C1F4F8881998125
:102AB000B801CBDA888199816FEF70E067DADF9136
:102AC000CF911F910F91FF900895EF92FF921F9366
:102AD000CF93DF937C01EC0110E0C7016E81412FA1
:102AE00023DF888599859F838E8322961F5F13310C
:102AF000A1F7DF91CF911F91FF90EF900895DF92A2
:102B0000EF92FF920F931F93CF93DF93EC01D62E9A
:102B1000842F6AE00E94AE35082F282F30E086EF20
:102B20009FEFBC01269FC001279F900D369F900DFF
:102B30001124840F911D62E070E00E94BA357B0180
:102B400010E017C0101728F4888199816FEF70E0AA
:102B500008C0101741F488819981E114F10429F02B
:102B6000B70114DA05C08881998165E571E046DA1C
:102B70001F5F1D1538F3DF91CF911F910F91FF90CB
:102B8000EF90DF900895CF92DF92EF92FF920F9334
:102B90001F93CF93DF938C016A01660F660F660F58
:102BA000C0E0D0E06064E62EFF24BE016E297F29DC
:102BB000F8018081918149DAF601EC0FFD1F6081F7
:102BC00070E0F80180819181E1D92196C830D1056A
:102BD00061F7DF91CF911F910F91FF90EF90DF9000
:102BE000CF900895CF92DF92EF92FF920F931F93B1
:102BF000CF93DF938C016A01660F660F660FC0E00A
:102C0000D0E06064E62EFF24BE016E297F29F80122
:102C1000808191811ADAF601EC0FFD1FE4916E2F8D
:102C200070E0F80180819181B1D92196C830D10539
:102C300059F7DF91CF911F910F91FF90EF90DF90A7
:102C4000CF9008950F931F938C0161E041ED51E007
:102C5000C9DFC80162E049ED51E0C4DFC80163E0AB
:102C600041EE51E0BFDFC80164E049EE51E0BADF58
:102C7000C80165E041EF51E0B5DFC80166E049EF0A
:102C800051E0B0DFC80167E041E052E0ABDF1F91E7
:102C90000F9108950F931F938C0161E041EB51E078
:102CA000A1DFC80162E049EB51E09CDFC80163E0AD
:102CB00041EC51E097DFC80164E049EC51E092DF5C
:102CC0001F910F9108950F931F938C0165E041E9C7
:102CD00051E088DFC80166E049E951E083DFC801BF
:102CE00067E041EA51E07EDFC80168E049EA51E06F
:102CF00079DF1F910F9108950F931F938C0165E069
:102D000041E751E06FDFC80166E049E751E06ADF63
:102D1000C80167E041E851E065DFC80168E049E8C3
:102D200051E060DF1F910F9108950F931F938C0165
:102D300061E041E551E056DFC80162E049E551E05C
:102D400051DFC80163E041E651E04CDFC80164E0B7
:102D500049E651E047DF1F910F9108950F931F93AC
:102D60008C0161E041E151E03DDFC80162E049E1F1
:102D700051E038DFC80163E041E251E033DFC801D0
:102D800064E049E251E02EDFC80165E041E351E033
:102D900029DFC80166E049E351E024DFC80167E0AC
:102DA00041E451E01FDFC80168E049E451E01ADF67
:102DB0001F910F9108950F931F938C0161E049EECD
:102DC00050E010DFC80162E041EF50E00BDFC801C6
:102DD00063E049EF50E006DFC80166E041E051E002
:102DE00001DFC80168E049E051E0FCDE1F910F916E
:102DF00008950F931F93CF93DF93EC01062F10E0FC
:102E000006C0888199816EEF70E0C0D81F5F1017EF
:102E1000C0F3DF91CF911F910F910895FF920F930F
:102E20001F93CF93DF93EC01162FCA01F22E6EA5EC
:102E30007FA54AE050E00E94FA39AEA5BFA5FD018A
:102E400001900020E9F73197EA1BFB0B0F2D0E1BB9
:102E5000CE01612FAD0153DD002329F0FF2019F0D1
:102E6000CE01602FC6DFDF91CF911F910F91FF90B0
:102E700008956F927F928F929F92AF92BF92CF925E
:102E8000DF92EF92FF920F931F93CF93DF937C011A
:102E9000A62EC42EDD2459E5652E51E0752E620E56
:102EA000711CF3018081B601680F711DF7018081EB
:102EB0009181CBD8CA2DD0E05E01AA0CBB1CAA0C14
:102EC000BB1C0DEA11E0F801EA0DFB1D608170E00A
:102ED000F701808191815AD845010894811C911C89
:102EE000F801E80DF91D608170E0F70180819181A2
:102EF0004DD8E50122960C0F1D1FF801608170E08E
:102F0000F7018081918142D8F3018181B601680F78
:102F1000711DF7018081918198D805ED11E0F801CC
:102F2000EA0DFB1D608170E0F701808191812ED850
:102F3000F801E80DF91D608170E0F7018081918151
:102F400025D80C0F1D1FF801608170E0F70180810A
:102F500091811CD8F3018281B601680F711DF701C0
:102F60008081918172D80DEF11E0F801EA0DFB1D0F
:102F7000608170E0F7018081918108D8F801E80D47
:102F8000F91D608170E0F701808191810E94C60F78
:102F90000C0F1D1FF801608170E0F70180819181A5
:102FA0000E94C60FF3018381C80ED11CF7018081F6
:102FB0009181B6014AD805E212E0A00EB11EF501DA
:102FC000608170E0F701808191810E94C60F800EC0
:102FD000911EF401608170E0F701808191810E946F
:102FE000C60F0C0F1D1FF801608170E0F701808192
:102FF00091810E94C60FDF91CF911F910F91FF9099
:10300000EF90DF90CF90BF90AF909F908F907F9088
:103010006F9008952F923F924F925F926F927F929E
:103020008F929F92AF92BF92CF92DF92EF92FF92D8
:103030000F931F935C01E62E642E7724F9E52F2E63
:10304000F1E03F2E220E311CF1018081B301680FA7
:10305000711DF501808191810E942510FF242701B7
:10306000440C551C440C551C7DE5C72E71E0D72E31
:10307000F601E40DF51D608170E0F501808191811C
:103080000E94C60F8701000F111F0E0D1F1D08940F
:10309000E11CF11C4701800E911EF601E80DF91D9F
:1030A000608170E0F501808191810E94C60F0894D3
:1030B000E11CF11CE00EF11ECE0CDF1CF60160815C
:1030C00070E0F501808191810E94C60FF10181813C
:1030D000680E711CF50180819181B3010E94251059
:1030E00005E811E0400E511EF201608170E0F5012B
:1030F000808191810E94C60F800E911EF401608133
:1031000070E0F501808191810E94C60F0E0D1F1D98
:10311000F801608170E0F501808191810E94C60F05
:103120001F910F91FF90EF90DF90CF90BF90AF90E5
:103130009F908F907F906F905F904F903F902F90D7
:1031400008952F923F924F925F926F927F928F924B
:103150009F92AF92BF92CF92DF92EF92FF920F9326
:103160001F93DF93CF93CDB7DEB76A970FB6F8946E
:10317000DEBF0FBECDBF6C015B01642E922E402ED0
:103180005E2C822F840F888F1A8293E69A8F198E75
:103190007724882410E01E010894211C311CB3E020
:1031A000EB2EF12CEC0EFD1E28C0AA0DBB1D8C9140
:1031B0008983112339F48D3229F473948394E1E0E7
:1031C000E98F0DC08E3221F08B3311F08C3239F43F
:1031D000F701E10FF11D808373941A8F0DC08053A6
:1031E0008A3050F4C1010E942739F701E10FF11D27
:1031F00080837394F4E08F0E1F5FA12FB0E0F50180
:1032000001900020E9F73197EA19FB09AE17BF07D3
:1032100060F2862D90E0881991091816190624F598
:10322000842D90E0A9E5EA2EA1E0FA2EE80EF91E21
:103230008C01050D111D075A1E4FA92CBB24962C7D
:1032400097180EC0F70181917F01B501680F711DBC
:10325000F601808191810E942510C601692DC9DD8A
:10326000E016F10679F76AC010E0F88D2F2E3324AE
:10327000E42CFF2489E591E0E80EF91E570108943B
:10328000A11CB11C57C01123E9F4998D9923D1F0E9
:10329000F60120813181692D70E0F4E05F1611F4B0
:1032A000F50101C0F7018081680F711DC9010E94FD
:1032B0002510F6018081918168E070E00E94C60FC0
:1032C000939437C0FA8D1F1781F4F6012081318164
:1032D000F4E05F1621F4C9016FEF70E003C0C9018B
:1032E00065E070E00E94C60F24C0892D90E003962F
:1032F00082159305F4F4E12FF0E082E0581661F4B2
:1033000083E090E08C0F9D1FE80FF91FC6016081DC
:10331000492D242D7FDE0BC083E090E08C0F9D1F94
:10332000E80FF91FC6016081492D242DA2DD94E02C
:10333000990E1F5F171508F4A6CF03C0988C981834
:1033400093CF6A960FB6F894DEBF0FBECDBFCF9174
:10335000DF911F910F91FF90EF90DF90CF90BF9082
:10336000AF909F908F907F906F905F904F903F9025
:103370002F900895CF92DF92EF92FF920F931F93B9
:103380006C01CB01142FF22EF60166A577A54AE059
:1033900050E00E94FA39F60166A577A5C601412FD3
:1033A0002F2DCFDE1F910F91FF90EF90DF90CF90E8
:1033B0000895FC01633008F062E06583E62FF0E0D9
:1033C000EA51FF4F6591749185E00C945A2DFC01F0
:1033D0008581833011F4158202C08F5F8583CF0110
:1033E0006581E7CFCF92DF92EF92FF920F931F9309
:1033F0008C016B019ADCC8017FDCC80162E0D9DF77
:1034000083E06FEF70E00E945A2D62E370E080E08D
:1034100090E00E94CC2C83E068E270E00E945A2D7C
:1034200062E370E080E090E00E94CC2C83E060E0FA
:1034300070E00E945A2DEE24D7FCE094FE2CC701C8
:10344000B6010E94CC2C1F910F91FF90EF90DF905E
:10345000CF9008956F927F928F929F92AF92BF927A
:10346000CF92DF92EF92FF920F931F93DF93CF9350
:10347000CDB7DEB76E970FB6F894DEBF0FBECDBFE7
:103480003B0169017A014801CA01B90120E030E03D
:1034900040E050E00E94243288232CF0C701B6019E
:1034A0000E946E3604C0C701B6010E945B360E94BE
:1034B000D4325B01B501882777FD8095982F0E9453
:1034C0007A329B01AC01C701B6010E94E02F7B015B
:1034D0008C01B401882777FD8095982F0E947A325D
:1034E0009B01AC01C801B7010E9432300E94D43266
:1034F0006B0177FF09C0D094C194D108D394A11473
:10350000B10411F441E001C040E0C4016AE070E0A0
:103510000E94BA357B0199242AE030E00EC0C21621
:10352000D3060CF49394C901880F991F13E0220F5E
:10353000331F1A95E1F7280F391FE216F3067CF7BF
:10354000442381F08DE28983C501BE016E5F7F4F08
:103550004AE050E00E94FA399E01205F3F4FF90196
:1035600090E306C0C501BE016F5F7F4FF1CF91931D
:103570008E2F821B8915D8F38E01005F1F4FB80173
:10358000690D711DC6014AE050E00E94FA39E00E53
:10359000F11EF7011082C301BE016F5F7F4F0E94D1
:1035A000B139C30167E571E00E949239C301B801E6
:1035B0000E9492396E960FB6F894DEBF0FBECDBF53
:1035C000CF91DF911F910F91FF90EF90DF90CF90FF
:1035D000BF90AF909F908F907F906F9008956F9263
:1035E0007F928F929F92AF92BF92CF92DF92EF9293
:1035F000FF920F931F935C013A014B01F22ED02EE4
:10360000FC0166A577A5A401930104E610E022DF82
:10361000F50166A577A5C5014F2D2D2D0E2DEC2C9E
:1036200090DD1F910F91FF90EF90DF90CF90BF90B2
:10363000AF909F908F907F906F900895AF92BF92C0
:10364000CF92DF92EF92FF920F931F937C015A016A
:103650006B018901FC0166A577A5A6019501FADE3B
:10366000F70166A577A5808191810E94FE0F1F91C9
:103670000F91FF90EF90DF90CF90BF90AF900895A3
:10368000AF92BF92CF92DF92EF92FF920F931F9370
:103690005C0169017A0170E0FC01808191810E94E6
:1036A0002510C501B701A6019801C8DF1F910F9130
:1036B000FF90EF90DF90CF90BF90AF9008950F9361
:1036C0001F9304E610E0DCDF1F910F91089524E6BC
:1036D00030E0B4CFDC011496EC911497F0E0319611
:1036E000EE0FFF1FEA0FFB1F80819181B2C0DC014A
:1036F0001496EC911497F0E03196EE0FFF1FEA0F4D
:10370000FB1F80819181C0C0FC018481882311F45A
:10371000148202C08F5F8483CF01E9CF0F931F9380
:10372000CF93DF93EC011C8282E08D8381E090E0F7
:103730000E94F4118C0164E070E00E940E0F198366
:10374000088385E190E00E9404379FA78EA78881B7
:1037500099810E945310FE0180E090E0178216824A
:103760000196329684319105C9F789E090E00E9474
:10377000F4118C01A0D11B830A83DF91CF911F919B
:103780000F910895FC0181E592E0918380838091FF
:103790006C0490916D049383828314821582168247
:1037A00017820895FC0181E592E0918380838091E6
:1037B0006C0490916D049383828314821582168227
:1037C00017820895FC0181E592E0918380837383E1
:1037D000628360E070E04483558366837783089555
:1037E000FC0181E592E0918380837383628360E0D2
:1037F00070E044835583668377830895FC01848158
:10380000982F937E8C71843011F4986001C094607D
:1038100094830895FC012581922F92959F703681A3
:10382000832F8295807F892B865F982F9295907F3A
:103830002F70292B2583982F92959F70307F392BDD
:1038400036838E3620F02F702583307F36831086A6
:103850000895CF93DF93EC0128859D8192959F7009
:103860008E818295807F892B281749F4E881F98120
:103870000280F381E02DCE010995188602C02F5FEA
:103880002887DF91CF910895CF93DF93EC018A8150
:103890009B810E9453108C8187FF03C08CE694E0CB
:1038A000F9D98D8181FF03C08CE694E0CBD98D815D
:1038B00080FF03C08CE694E006DA8D8183FF03C0AD
:1038C0008CE694E078DA8D8182FF03C08CE694E088
:1038D00045DA8C81817080939D048C8186958170FE
:1038E00080939E048C8182958695837080939C043E
:1038F0009D8192959F708E818295807F892B88878C
:10390000E881F9810190F081E02DCE010995DF91E8
:10391000CF910895FC0189E592E091838083089519
:10392000FC0189E592E0918380830895EF92FF92F4
:103930001F93FC018281938165E870E00E9425104D
:103940008CE6E82E84E0F82E409112045091130486
:10395000C70165E823E062DA4091EA035091EB0386
:10396000C70160E924E05ADA60915A016B5F209147
:103970000604309107044091080450910904C701DE
:103980009EDE60915A01605F20910A0430910B0421
:1039900040910C0450910D04C70191DE60915B01D0
:1039A0006C5F4091220450912304C70124E036DA71
:1039B00060915B01625F2091FE033091FF034091B3
:1039C000000450910104C7017ADE10915C018FE080
:1039D0000E943F2EAC01C701612F21E01FDA109138
:1039E0005C011B5F6091E60470E080E090E00E9463
:1039F00025339B01AC01C701612F61DE10915C0191
:103A0000175F6091E70470E080E090E00E9425334A
:103A10009B01AC01C701612F52DE60915C01635FC5
:103A20002091DD043091DE044091DF045091E004E8
:103A3000C70145DE1F91FF90EF9008950F931F93EC
:103A40008C01FC0182819381609159014CE152E02B
:103A50000E94431060915901665FF8018281938151
:103A600047E152E00E944310F80182819381609106
:103A70005A0142E152E00E944310F8018281938191
:103A800060915B014EE052E00E94431060915B0147
:103A9000665FF8018281938149E052E00E94431001
:103AA0001F910F910895FC0189E592E09183808335
:103AB000CF010C94EF110F931F938C0163DE89E506
:103AC00092E0F8019183808394819C718681807F4C
:103AD00086839364948384EA85831F910F9108956C
:103AE0000F931F938C014EDE89E592E0F8019183DC
:103AF000808394819C718681807F86839364948384
:103B000084EA85831F910F910895FC011486138622
:103B100088E893E1928781870895FC018481282FAA
:103B2000269526952F5F2770922F990F990F837EE8
:103B3000892B848330E0263031051CF0837E84603D
:103B400084830895AF92BF92CF92DF92EF92FF925B
:103B50000F931F93CF93DF93EC018C81869586950D
:103B6000877090E08330910539F18430910534F409
:103B70008130910559F0029731F412C084309105DB
:103B800051F00597F1F020E030E01FC02091BE0316
:103B90003091BF031AC0209112043091130415C054
:103BA000609118047091190480911A0490911B047B
:103BB0000E94D4329B0109C020911004309111045D
:103BC00004C020910E0430910F0489859A8528172E
:103BD000390714F43A8729878B859C8582179307C8
:103BE00014F43C872B8700D000D0B901882777FDDB
:103BF0008095982F29853A85442737FD4095542F85
:103C0000EB84FC840027F7FC0095102FE1E2AE2E38
:103C1000B12CC12CD12CEDB7FEB7A182B282C382E8
:103C2000D482AA24BB246501D7D50F900F900F90A2
:103C30000F906132710514F060E270E08B0177FF44
:103C400002C000E010E08CE694E0602F43E10E94A7
:103C5000941410939904009398048CE694E00E94C5
:103C600065154C8146954695477050E08CE694E08A
:103C700060E820E0D3D88A819B8161E672E00E94EF
:103C8000FE0F488550E08CE694E060E020E0C6D866
:103C90004091A4045091A5046091A6047091A704DA
:103CA00080E995E02AE030E064D4DF91CF911F9164
:103CB0000F91FF90EF90DF90CF90BF90AF9008955D
:103CC0000F931F938C015EDD87E692E0F8019183EC
:103CD000808395818681807F868384E08483987049
:103CE000926A95831F910F9108950F931F938C01F2
:103CF00049DD87E692E0F801918380839581868192
:103D0000807F868384E084839870926A95831F9174
:103D10000F910895FC0181858F5F8187843008F0C1
:103D200011860895CF93DF93EC01498550E08CE62E
:103D300094E064E820E072D88A819B8163EC70E0B3
:103D40000E942510E985F0E0EE0FFF1FEE0FFF1F28
:103D5000EC5CFB4F608171818281938120E030E0D7
:103D600040E050E00E944F322A813B81882324F4B6
:103D7000C9016BE672E003C0C9016DE672E00E9402
:103D8000FE0FE985F0E0EE0FFF1FEE0FFF1FEC5C6A
:103D9000FB4F60817181828193810E94D4329B01AB
:103DA00077FF03C0309521953F4FB901882777FDF4
:103DB0008095982F0E947A32AB01BC018CE694E08A
:103DC00086DCE985F0E0EE0FFF1FEE0FFF1FEC5BD6
:103DD000FB4F408151818CE694E06EEC20E01ED8D0
:103DE000E985F0E0EE0FFF1FEE0FFF1FEC5AFB4FCF
:103DF00060817181828193810E94D4329B01AC01E8
:103E00008CE694E068E9A90120E008D8E985F0E0B3
:103E1000EE0FFF1FE45DFB4F408151818CE694E083
:103E200062EA20E00E940E17DF91CF9108950F9370
:103E30001F938C01FC018281938160E84FE352E083
:103E40000E944310F8018281938160EC40E352E0CC
:103E50000E944310F8018281938164E941E252E0BB
:103E60000E9443101F910F9108950F931F938C018F
:103E700089DC83E792E0F8019183808394819C71CF
:103E8000258128708681807F868393649483206255
:103E9000258311861F910F9108950F931F938C0115
:103EA00071DC83E792E0F8019183808394819C71B7
:103EB000258128708681807F868393649483206225
:103EC000258311861F910F9108951F920F920FB6AF
:103ED0000F9211242F933F934F938F939F93EF93C0
:103EE000FF934091C600E0918C05F0918D053196CD
:103EF0009F012F773070319780918E0590918F05BB
:103F00002817390739F0E45FFA4F408330938D0565
:103F100020938C05FF91EF919F918F914F913F914D
:103F20002F910F900FBE0F901F9018958F92AF9208
:103F3000CF92DF92EF92FF920F931F93DF93CF9375
:103F4000CDB7DEB7FC018BE792E09183808373836A
:103F50006283558344833783268311870087F386E2
:103F6000E286D586C486A68687868D85808B8E85DB
:103F7000818B8F85828BCF91DF911F910F91FF9065
:103F8000EF90DF90CF90AF908F9008958F92AF9287
:103F9000CF92DF92EF92FF920F931F93DF93CF9315
:103FA000CDB7DEB7FC018BE792E09183808373830A
:103FB0006283558344833783268311870087F38682
:103FC000E286D586C486A68687868D85808B8E857B
:103FD000818B8F85828BCF91DF911F910F91FF9005
:103FE000EF90DF90CF90AF908F900895CF93DF93B5
:103FF000EC019A01AB01E885F985203081EE3807A4
:1040000080E0480780E0580709F445C081E090E06F
:104010000A8802C0880F991F0A94E2F7808360E043
:1040200079E08DE390E00E94CD3521503040404052
:1040300050405695479537952795EC81FD81308303
:10404000EE81FF812083EA85FB85208141E050E0FD
:10405000CA010E8402C0880F991F0A94E2F7282B28
:104060002083EA85FB852081CA010F8402C0880F66
:10407000991F0A94E2F7282B2083EA85FB8580812B
:10408000088802C0440F551F0A94E2F7842B8083EE
:10409000DF91CF910895108220E130E0CECFFC0176
:1040A000A285B3854C9121E030E0C901068402C0AD
:1040B000880F991F0A94E2F7809584238C93A28538
:1040C000B3854C91C901078402C0880F991F0A94D7
:1040D000E2F7809584238C93A285B3858C91008828
:1040E00002C0220F331F0A94E2F7209528232C9355
:1040F0000895DC011296ED91FC911397E058FF4F63
:104100002191319180819181281B390B2F7730705B
:10411000C9010895DC011296ED91FC911397EE57B9
:10412000FF4F2081318192918291E058F0408217B7
:10413000930719F42FEF3FEF05C0E20FF31F8081C3
:10414000282F30E0C9010895DC011296ED91FC9111
:104150001397DF01AE57BF4F2D913C911197E05857
:10416000FF4F80819181E058F0408217930719F446
:104170002FEF3FEF0BC0E20FF31F80812F5F3F4F08
:104180002F7730702D933C93282F30E0C90108958C
:10419000DC011296ED91FC911397EE57FF4F808151
:1041A0009181929382930895FC01A085B185218924
:1041B0008C9190E0022E02C0959587950A94E2F7C3
:1041C00080FFF6CF0484F585E02D608308958BE7AA
:1041D00092E090939105809390058CE095E0909308
:1041E00093058093920585EC90E0909395058093DC
:1041F000940584EC90E0909397058093960580EC6D
:1042000090E0909399058093980581EC90E09093CD
:104210009B0580939A0586EC90E090939D05809392
:104220009C0584E080939E0583E080939F0587E052
:104230008093A00585E08093A10581E08093A2058D
:1042400008950F931F93CF93DF938C01EB0109C067
:104250002196D801ED91FC910190F081E02DC801EB
:10426000099568816623A1F7DF91CF911F910F9186
:104270000895EF92FF920F931F93CF93DF938C01DA
:104280007B01EA010CC0D7016D917D01D801ED9150
:10429000FC910190F081E02DC801099521972097AC
:1042A00091F7DF91CF911F910F91FF90EF900895BB
:1042B000DC01ED91FC910280F381E02D09950895D8
:1042C000CF92DF92EF92FF920F931F93CF93DF93E2
:1042D0006C017B01C0E0D0E00DC0D601ED91FC91F6
:1042E00000811181C701BE013DD3682FC601F801CD
:1042F00009952196F70184819581C817D90768F33C
:10430000DF91CF911F910F91FF90EF90DF90CF90B1
:1043100008952F923F924F925F926F927F928F9269
:104320009F92AF92BF92CF92DF92EF92FF920F9344
:104330001F93DF93CF93CDB7DEB7A0970FB6F89456
:10434000DEBF0FBECDBF1C016A017B0141155105C7
:104350006105710541F440E350E060E070E020E069
:1043600030E09BD053C0882499245401422E552418
:104370006624772401E010E00C0F1D1F080D191DA5
:10438000C701B601A30192010E94CD35F8016083F7
:104390000894811C911CA11CB11CC701B601A3018A
:1043A00092010E94CD35C901DA016C017D01C11471
:1043B000D104E104F104F1F681E0E82EF12CEC0ED9
:1043C000FD1EE80CF91C3E010894611C711CD5010E
:1043D000C4010197A109B1096C01C818D90813C01B
:1043E000F601EE0DFF1D40814A3010F4405D01C022
:1043F000495C50E060E070E0C10120E030E04DD069
:104400000894E108F1086E147F0451F7A0960FB6E6
:10441000F894DEBF0FBECDBFCF91DF911F910F91FA
:10442000FF90EF90DF90CF90BF90AF909F908F90D4
:104430007F906F905F904F903F902F900895DC0198
:104440002115310541F4ED91FC910190F081E02DB1
:10445000642F099508955DCFEF92FF920F931F93FC
:104460009A017B0100E010E0B801A701E8DF1F918D
:104470000F91FF90EF900895EF92FF920F931F938B
:104480009A01E62EFF2400E010E0B801A701D7DF73
:104490001F910F91FF90EF900895EF92FF920F936D
:1044A0001F93CF93DF93EC017A018B012115310526
:1044B00041F4E881F9810190F081E02D642F0995A4
:1044C00019C02A303105A9F477FF0FC04DE250E042
:1044D00060E070E020E030E0E0DF10950095F094BF
:1044E000E094E11CF11C011D111DCE01B801A701D2
:1044F0002AE00FDFDF91CF911F910F91FF90EF9096
:104500000895EF92FF920F931F937B019A0100276A
:10451000F7FC0095102FB801A701BFDF1F910F9185
:10452000FF90EF900895EF92FF920F931F939A01DF
:10453000E62EFF2400E010E0B801A701AEDF1F91D6
:104540000F91FF90EF9008950F931F938C014DE012
:1045500050E060E070E020E030E09FDFC8014AE01A
:1045600050E060E070E020E030E097DF1F910F91B5
:1045700008950F931F938C0162DFC801E5DF1F913F
:104580000F910895CF92DF92EF92FF920F931F93B6
:104590008C019A016B01EE24FF24B701A6014FDFC5
:1045A000C801D2DF1F910F91FF90EF90DF90CF9065
:1045B0000895CF92DF92EF92FF920F931F938C0199
:1045C0009A01C62EDD24EE24FF24B701A60137DFB1
:1045D000C801BADF1F910F91FF90EF90DF90CF904D
:1045E00008950F931F938C0163DEC801ADDF1F9107
:1045F0000F9108950F931F93CF93DF938C01EB01DD
:104600000AC02196F901449150E060E070E0C801D1
:1046100020E030E014DF9E01FE018491882389F7B9
:10462000C80192DFDF91CF911F910F9108950F93F1
:104630001F938C0145DEC80187DF1F910F910895FC
:104640000F931F938C0129DFC8017EDF1F910F910B
:104650000895CF92DF92EF92FF920F931F938C01F8
:104660006B019A01EE24D7FCE094FE2CB701A60161
:1046700014DFC80169DF1F910F91FF90EF90DF9069
:10468000CF900895CF92DF92EF92FF920F931F93F6
:104690008C019A01C62EDD24EE24FF24B701A60169
:1046A000FCDEC80151DF1F910F91FF90EF90DF906A
:1046B000CF9008959F92AF92BF92CF92DF92EF92E8
:1046C000FF920F931F93CF93DF93EC017A018B013D
:1046D000922ECB01BA0120E030E040E050E00E9491
:1046E0004F32882364F4CE014DE250E060E070E088
:1046F00020E030E0D2DE17FB109517F9109520E08E
:1047000030E040E05FE3AA240BC0CA01B90120E019
:1047100030E040E251E40E9427319B01AC01A394B8
:10472000A91498F3C801B7010E940B305B016C011A
:104730000E946E2E7B018C01CE01B801A7012AE0F8
:1047400030E07DDE992021F0CE016BE972E0B0DD32
:10475000C801B7010E9425339B01AC01C601B50118
:104760000E94E02F21C020E030E040E251E40E94AE
:1047700032307B018C010E94D4325B016C01CC246D
:10478000B7FCC094DC2CCE01B601A5012AE030E0D4
:1047900084DEC601B5010E947A329B01AC01C801DA
:1047A000B7010E94E02F9A949920E9F6DF91CF910A
:1047B0001F910F91FF90EF90DF90CF90BF90AF903F
:1047C0009F90089577CF0F931F938C0173DFC801DB
:1047D000BBDE1F910F9108952F923F924F925F92EF
:1047E0006F927F928F929F92AF92BF92CF92DF9201
:1047F000EF92FF920F931F93DF93CF93CDB7DEB766
:104800003B014C0119012A016D897E898F89988DA0
:104810006A197B098C099D09621A730A840A950A30
:10482000A40193010E948F35E218F30804091509C9
:10483000A80197010E94EF352A0D3B1D4C1D5D1DFF
:10484000B901CA01CF91DF911F910F91FF90EF90B5
:10485000DF90CF90BF90AF909F908F907F906F90A0
:104860005F904F903F902F900895089570E0382FFB
:1048700020E0622B732BCB010895EF92FF920F93F0
:104880001F937B018C01611571058105910529F448
:1048900020E030E040E050E00BC00E945438A80116
:1048A00097010E94EF35AC01CB01DA019C01AD010B
:1048B000B901CA011F910F91FF90EF900895EF92F7
:1048C000FF920F931F937B018C016217730784077C
:1048D00095075CF4261B370B480B590BCA01B9012D
:1048E000CCDFE60EF71E081F191FB701C8011F9184
:1048F0000F91FF90EF900895009729F0BC0180E0A0
:1049000090E00C9457380895FC010190F081E02D5F
:10491000E60FF71F80810895DC01ED91FC9111975E
:10492000309751F014968D919C91159768177907DF
:1049300018F4E60FF71F40830895FC019B01848162
:1049400095816817790728F4608171816115710577
:1049500029F41092A30563EA75E002C0620F731F89
:10496000CB010895FC010190F081E02DE60FF71FC7
:1049700080810895FC01808191810C9444390F93CA
:104980001F93CF93DF93FC018B0141155105A1F0DB
:104990006115710589F084819581EA0121978C1751
:1049A0009D0708F4EC0160817181C801AE010E948D
:1049B000C639C00FD11F1882DF91CF911F910F917F
:1049C00008950F931F93CF93DF93FC018B01411543
:1049D0005105A1F06115710589F084819581EA0185
:1049E00021978C179D0708F4EC0160817181C80143
:1049F000AE010E94C639C00FD11F1882DF91CF913E
:104A00001F910F9108950F931F938C01FC018081DA
:104A100091810E94B137F8011382128215821482AB
:104A20001F910F910895FC01DB0114962D913C918B
:104A3000159784819581821B930B8417950710F439
:104A400080E00895808191816D917C91840F951F04
:104A5000A9010E94B8399C0180E0232B09F481E070
:104A60000895FC01DB012481358114968D919C9180
:104A700015972817390710F480E00895CF0140E01A
:104A800050E0D1CFDF92EF92FF920F931F93CF931D
:104A9000DF93EC018C819D8148175907B8F47A01A6
:104AA0000894E11CF11CE881F981EE0DFF1DD08016
:104AB000108208811981C80170E00E94D5399C01DB
:104AC0000E0D1F1DF801D082009719F4EFEFFFEFD4
:104AD00005C088819981F901E81BF90BCF01DF91AD
:104AE000CF911F910F91FF90EF90DF900895FC01FF
:104AF0004481558141505040C5CFCF93DF93FC0195
:104B0000DB01848195814817590760F4C081D18108
:104B10006D917C91CE01840F951F0E94E0399C011C
:104B2000009719F42FEF3FEF02C02C1B3D0BC9017A
:104B3000DF91CF91089540E050E0DFCFCF93DF9336
:104B4000FC01848195814817590758F4C081D181AF
:104B5000CE01840F951F70E00E949D399C01009743
:104B600019F42FEF3FEF02C02C1B3D0BC901DF9161
:104B7000CF91089540E050E0E1CFDC01FB011496B5
:104B80002D913C911597848195812817390711F053
:104B900080E00895608171818D919C910E94A83977
:104BA0009C0180E0232B09F481E00895FC01DB01E6
:104BB0002481358114968D919C911597281739077A
:104BC00010F480E00895281B390B808191816D914C
:104BD0007C91820F931F0E94A8399C0180E0232BB7
:104BE00009F481E00895DC01FB01608171818D9100
:104BF0009C910E94A839292F332727FD30952095B5
:104C000030952227330F221F3327C9010895DC0175
:104C1000FB01608171818D919C910E94A83940E0D7
:104C200050E01816190614F041E050E0CA0108954A
:104C3000DC01FB01608171818D919C910E94A839FA
:104C400040E050E01816190614F441E050E0CA01A3
:104C50000895DC01FB01608171818D919C910E941E
:104C6000A839292F332727FD30952227330F221FFC
:104C70003327C9010895DC01FB0114962D913C9165
:104C80001597848195812817390751F460817181C6
:104C90008D919C910E94A8399C0180E0232B09F002
:104CA00081E090E00895DC01FB0114962D913C9188
:104CB0001597848195812817390711F080E00BC082
:104CC000608171818D919C910E94A8399C0180E046
:104CD000232B09F481E090E00895FC01DB016D9144
:104CE0007C91808191810C94A8390F931F93CF936D
:104CF000DF93EC018B01FB01648175818C819D81C7
:104D0000680F791F7D836C838A819B818617970743
:104D1000B8F46F5F7F4F888199810E9460384C8121
:104D20005D81009729F0998388835B834A8308C05B
:104D3000F80184819581481B590B5D834C8307C022
:104D4000F80160817181888199810E949239CE0138
:104D5000DF91CF911F910F910895C7CFCF93DF932C
:104D6000EC01CB017B836A8301960E94043799830F
:104D70008883009721F41B821A821D821C82DF9196
:104D8000CF9108950F931F93CF93DF93EC018B0185
:104D90008617970701F1FB01248135818C819D8164
:104DA0008217930748F4888199810E94B137F801EE
:104DB00064817581CE01D2DF2881398121153105C9
:104DC00051F0F801848195819D838C83608171818C
:104DD000C9010E94B139CE01DF91CF911F910F918E
:104DE00008951F93CF93DF93EC01162F81E090E09D
:104DF0009D838C83CE0161E070E0B0DFE881F981B2
:104E0000309721F01083E881F9811182DF91CF91F1
:104E10001F9108951F93CF93DF93EC01162F81E02C
:104E200090E09D838C83CE0161E070E097DFE881A4
:104E3000F981309721F01083E881F9811182DF91A7
:104E4000CF911F9108951F93CF93DF93EC01162FFD
:104E500081E090E09D838C83CE0161E070E07EDF95
:104E6000E881F981309721F01083E881F98111827E
:104E7000DF91CF911F9108951F93CF93DF93EC01A2
:104E8000162F81E090E09D838C83CE0161E070E07D
:104E900065DFE881F981309721F01083E881F9819D
:104EA0001182DF91CF911F9108950F931F93CF939C
:104EB000DF938C01EB016C817D81FC017583648340
:104EC0004DDFF80180819181009721F0688179811F
:104ED0000E94B139DF91CF911F910F9108950F93E7
:104EE0001F93CF93DF938C01EB016C817D81FC01DB
:104EF0007583648333DFF80180819181009721F00D
:104F0000688179810E94B139DF91CF911F910F9112
:104F10000895EF92FF920F931F93DF93CF93CDB736
:104F2000DEB7A1970FB6F894DEBF0FBECDBF8C01E0
:104F3000CB01BA017E010894E11CF11CA7012AE013
:104F400030E00E94683AF70101900020E9F73197BC
:104F5000EE19FF09D8011596FC93EE931497C8013A
:104F6000BF01FCDEF80180819181009719F0B70143
:104F70000E94B139A1960FB6F894DEBF0FBECDBF27
:104F8000CF91DF911F910F91FF90EF900895EF92D5
:104F9000FF920F931F93DF93CF93CDB7DEB7A19707
:104FA0000FB6F894DEBF0FBECDBF8C01CB01BA01A6
:104FB0007E010894E11CF11CA7012AE030E00E9468
:104FC000683AF70101900020E9F73197EE19FF09DF
:104FD000D8011596FC93EE931497C801BF01BEDE6D
:104FE000F80180819181009719F0B7010E94B139D1
:104FF000A1960FB6F894DEBF0FBECDBFCF91DF9163
:105000001F910F91FF90EF900895EF92FF920F93F1
:105010001F93DF93CF93CDB7DEB7A1970FB6F89468
:10502000DEBF0FBECDBF8C019A0180E090E07E0113
:105030000894E11CF11CA7010E94683AF701019055
:105040000020E9F73197EE19FF09D8011596FC9376
:10505000EE931497C801BF0181DEF8018081918130
:10506000009719F0B7010E94B139A1960FB6F894D4
:10507000DEBF0FBECDBFCF91DF911F910F91FF908B
:10508000EF900895EF92FF920F931F93DF93CF93CA
:10509000CDB7DEB7A1970FB6F894DEBF0FBECDBF78
:1050A0008C019A0180E090E07E010894E11CF11CE3
:1050B000A7010E94683AF70101900020E9F73197B3
:1050C000EE19FF09D8011596FC93EE931497C801C9
:1050D000BF0144DEF80180819181009719F0B7018A
:1050E0000E94B139A1960FB6F894DEBF0FBECDBFB6
:1050F000CF91DF911F910F91FF90EF9008950F9343
:105100001F93CF93DF938C01EB016115710511F4AF
:10511000C7EAD2E0FE0101900020E9F73197EC1BCD
:10512000FD0BD8011596FC93EE931497C801BF01AF
:1051300015DEF80180819181009719F0BE010E946F
:10514000B139DF91CF911F910F910895AF92BF9226
:10515000CF92DF92EF92FF920F931F93CF93DF9343
:10516000B82EA92E6B01C82FD92FFB016081718148
:10517000CE01C5DFEE24FF240EC0088119810E0D7B
:105180001F1DF801808190E00E947A39F801808328
:105190000894E11CF11CF60184819581E816F9065A
:1051A00060F38B2D9A2DDF91CF911F910F91FF907E
:1051B000EF90DF90CF90BF90AF900895AF92BF92E5
:1051C000CF92DF92EF92FF920F931F93CF93DF93D3
:1051D000B82EA92E6B01C82FD92FFB0160817181D8
:1051E000CE018DDFEE24FF240EC0088119810E0D43
:1051F0001F1DF801808190E00E947239F8018083C0
:105200000894E11CF11CF60184819581E816F906E9
:1052100060F38B2D9A2DDF91CF911F910F91FF900D
:10522000EF90DF90CF90BF90AF900895EF92FF92F4
:105230000F931F93DF93CF93CDB7DEB72C970FB6A5
:10524000F894DEBF0FBECDBFFC017B018617970728
:1052500011F401E025C024813581DB0114968D9184
:105260009C9115972817390711F000E019C0CE015D
:105270000196BF01A3DF09811A81CE010796B7010C
:105280009DDF6F817885C8010E94A83900E00097F2
:1052900009F401E0CE010796B6DBCE010196B3DB3F
:1052A000802F2C960FB6F894DEBF0FBECDBFCF91E6
:1052B000DF911F910F91FF90EF900895CF92DF92B1
:1052C000EF92FF921F93CF93DF936C017B01B901A3
:1052D0002417350710F4BA01A901D70114968D914E
:1052E0009C911597EB018617970708F4EC01D701FD
:1052F000ED91FC911197EC0FFD1F108110826D91C3
:105300007C91640F751FC601FADED701ED91FC9107
:10531000EC0FFD1F1083C601DF91CF911F91FF900D
:10532000EF90DF90CF9008950F931F938C01FB01B6
:1053300024813581C3DFC8011F910F9108958F9299
:105340009F92AF92BF92CF92DF92EF92FF920F9314
:105350001F93DF93CF9300D000D000D0CDB7DEB73E
:105360005C016B01DB0114968D919C911597009760
:1053700089F101974817590768F1F50184819581F2
:105380004817590738F5ED91FC9100817A014E01DB
:105390000894811C911C1CC0D501ED91FC91EE0D6F
:1053A000FF1D8081801789F4F601248135812E0D3F
:1053B0003F1DC401B501A70181DFC401B601DDDBDA
:1053C000182FC40120DB112341F40894E108F108EF
:1053D000F7FEE2CFEE24EA94FE2CC70126960FB624
:1053E000F894DEBF0FBECDBFCF91DF911F910F911B
:1053F000FF90EF90DF90CF90BF90AF909F908F90F5
:105400000895FC01DB014481558114968D919C9196
:105410001597481B590BCF0192CFAF92BF92CF92F5
:10542000DF92EF92FF920F931F93DF93CF9300D001
:1054300000D000D0CDB7DEB75C018B01DB016D91F0
:105440007C916115710519F4B8012FDD3BC0CE01C7
:10545000019655DEF801E480F580CC24DD240EC0F1
:10546000D801ED91FC91EC0DFD1D808190E00E9432
:105470006A39892B31F00894C11CD11CCE14DF0489
:1054800078F3ED80FE800BC0D801ED91FC91EE0D1C
:10549000FF1D808190E00E946A39892B31F00894C9
:1054A000E108F108CE14DF0478F30894E11CF11C44
:1054B000C5018E010F5F1F4FB801A6019701FEDEE7
:1054C000C801A1DAC50126960FB6F894DEBF0FBE5B
:1054D000CDBFCF91DF911F910F91FF90EF90DF90A3
:1054E000CF90BF90AF9008952F923F924F925F92CE
:1054F0006F927F928F929F92AF92BF92CF92DF92E4
:10550000EF92FF920F931F93DF93CF93CDB7DEB748
:1055100068970FB6F894DEBF0FBECDBF3C01FB010C
:105520002A011901608171816115710519F4BF01AA
:10553000BCDC4CC07E010894E11CF11CC701DFDD1E
:105540008E01095F1F4FC80167EA72E0D8DDD02ED7
:10555000C12E3DE0832E912C8C0E9D1E23E1A22EA8
:10556000B12CAC0EBD1E1DC0C401B70140E050E01F
:105570009801A4DE8D2D9C2DB401B7DBC40143DA64
:105580008D2D9C2DB101B1DBF20144815581400F7D
:10559000511FC501B701C8DEC701B501F3DBC50165
:1055A00032DAC701B201C7DA8C01FFEF8F3F9F07E4
:1055B000D9F68D2D9C2DB70198DBC3016D2D7C2D67
:1055C00074DC8D2D9C2D1FDAC7011DDAC30168968E
:1055D0000FB6F894DEBF0FBECDBFCF91DF911F9104
:1055E0000F91FF90EF90DF90CF90BF90AF909F9082
:1055F0008F907F906F905F904F903F902F90089585
:10560000EF92FF920F931F93DF93CF9300D000D0C0
:1056100000D0CDB7DEB77C01FB01142F022F6081D3
:1056200071816115710519F4BF013FDC16C0CE010F
:10563000019665DD89819A8101C00083612F70E048
:105640000E949D39FC010097C1F7C7018E010F5FD1
:105650001F4FB8012ADCC801D6D9C70126960FB65C
:10566000F894DEBF0FBECDBFCF91DF911F910F9198
:10567000FF90EF9008950F931F93CF93DF938C01CA
:10568000EB016115710511F4C7EAD2E0FE0101904A
:105690000020E9F73197EC1BFD0BD8011596FC9320
:1056A000EE931497C801BF0159DBF8018081918105
:1056B000009719F0BE010E94B139DF91CF911F917F
:1056C0000F910895EF92FF920F931F93DF93CF9363
:1056D000CDB7DEB7A1970FB6F894DEBF0FBECDBF32
:1056E0008C01CB01BA017E010894E11CF11CA701D9
:1056F0000E94193AF70101900020E9F73197EE195D
:10570000FF09D8011596FC93EE931497C801BF01C9
:1057100025DBF80180819181009719F0B7010E9483
:10572000B139A1960FB6F894DEBF0FBECDBFCF91B1
:10573000DF911F910F91FF90EF900895EF92FF92EC
:105740000F931F93DF93CF93CDB7DEB7A1970FB61B
:10575000F894DEBF0FBECDBF8C01CB01BA017E0134
:105760000894E11CF11CA7010E94193AF70101906D
:105770000020E9F73197EE19FF09D8011596FC933F
:10578000EE931497C801BF01E9DAF8018081918195
:10579000009719F0B7010E94B139A1960FB6F8949D
:1057A000DEBF0FBECDBFCF91DF911F910F91FF9054
:1057B000EF900895EF92FF920F931F93DF93CF9393
:1057C000CDB7DEB7A1970FB6F894DEBF0FBECDBF41
:1057D0008C01CB017E010894E11CF11CB7010E94F1
:1057E000FA39F70101900020E9F73197EE19FF0926
:1057F000D8011596FC93EE931497C801BF01AEDA59
:10580000F80180819181009719F0B7010E94B139A8
:10581000A1960FB6F894DEBF0FBECDBFCF91DF913A
:105820001F910F91FF90EF900895EF92FF920F93C9
:105830001F93DF93CF93CDB7DEB7A1970FB6F89440
:10584000DEBF0FBECDBF8C01CB017E010894E11CF1
:10585000F11CB7010E94FA39F70101900020E9F725
:105860003197EE19FF09D8011596FC93EE93149722
:10587000C801BF0173DAF80180819181009719F0A6
:10588000B7010E94B139A1960FB6F894DEBF0FBEE2
:10589000CDBFCF91DF911F910F91FF90EF900895B1
:1058A0001F920F920FB60F9211242F933F938F9355
:1058B0009F93AF93BF938091A8059091A905A09164
:1058C000AA05B091AB053091AC050196A11DB11DA3
:1058D000232F2D5F2D3720F02D570196A11DB11DCF
:1058E0002093AC058093A8059093A905A093AA05E1
:1058F000B093AB058091A4059091A505A091A60554
:10590000B091A7050196A11DB11D8093A4059093A8
:10591000A505A093A605B093A705BF91AF919F9150
:105920008F913F912F910F900FBE0F901F90189560
:105930008FB7F8942091A8053091A9054091AA0548
:105940005091AB058FBFB901CA0108959FB7F89474
:105950002091A4053091A5054091A6055091A70579
:1059600086B5A89B06C08F3F21F02F5F3F4F4F4F5A
:105970005F4F9FBF542F432F322F2227280F311DF7
:10598000411D511D82E0220F331F441F551F8A9570
:10599000D1F7B901CA010895EF92FF920F931F93B7
:1059A000CF93DF937B018C01D1DFEB010DC0CEDF04
:1059B0006C1B7D0B685E7340D0F30894E108F1081E
:1059C00001091109C851DC4FE114F1040105110569
:1059D00071F7DF91CF911F910F91FF90EF90089594
:1059E000019739F0880F991F880F991F0297019727
:1059F000F1F70895789484B5826084BD84B58160A0
:105A000084BD85B5826085BD85B5816085BDEEE6C6
:105A1000F0E0808181608083E1E8F0E010828081A5
:105A200082608083808181608083E0E8F0E0808113
:105A300081608083E1EBF0E0808184608083E0EB33
:105A4000F0E0808181608083EAE7F0E0808184601B
:105A50008083808182608083808181608083808177
:105A6000806880831092C10008958093A8020895F1
:105A7000982F8E3008F09E5097708091A8028295E2
:105A8000880F880F807C892B80937C0080917A001E
:105A9000806480937A0080917A0086FDFCCF20910B
:105AA000780040917900942F80E030E0282B392B4A
:105AB000C90108951F93CF93DF93182FEB0161E085
:105AC00057D0209709F44AC0CF3FD10509F449C007
:105AD000E12FF0E0E657FD4F84918330C1F0843030
:105AE00028F4813051F08230B1F50CC0863019F1C4
:105AF000873049F1843079F514C084B5806884BD5D
:105B0000C7BD32C084B5806284BDC8BD2DC0809140
:105B10008000806880938000D0938900C0938800C3
:105B200023C080918000806280938000D0938B009E
:105B3000C0938A0019C08091B00080688093B00043
:105B4000C093B30011C08091B00080628093B00018
:105B5000C093B40009C0C038D1051CF4812F60E0A7
:105B600002C0812F61E057D0DF91CF911F9108953E
:105B7000482F50E0CA018A589D4FFC0124914E598C
:105B80005D4FFA0184918823C1F0E82FF0E0EE0F19
:105B9000FF1FEC5BFD4FA591B491662341F49FB7C5
:105BA000F8948C91209582238C939FBF08959FB782
:105BB000F8948C91822B8C939FBF0895833071F061
:105BC000843028F48130A1F0823021F514C0863071
:105BD000B1F08730D1F08430E9F404C080918000C6
:105BE0008F7703C0809180008F7D8093800008951F
:105BF00084B58F7702C084B58F7D84BD0895809170
:105C0000B0008F778093B00008958091B0008F7DB1
:105C10008093B0000895FF920F931F93F62E482FA4
:105C200050E0CA0186579D4FFC012491CA018A5851
:105C30009D4FFC0114914E595D4FFA0104910023D0
:105C4000D1F0222311F0822FB9DFE02FF0E0EE0F28
:105C5000FF1FE25BFD4FA591B491FF2031F49FB788
:105C6000F8948C911095812304C09FB7F8948C917F
:105C7000812B8C939FBF1F910F91FF9008950F93DD
:105C80001F93482F50E0CA0186579D4FFC01249175
:105C9000CA018A589D4FFC0104914E595D4FFA018B
:105CA0001491112319F420E030E014C0222311F0E4
:105CB000822F84DF812F90E0880F991F885A9D4F93
:105CC000FC01A591B4918C9120E030E0802311F08B
:105CD00021E030E0C9011F910F910895EF92FF92EA
:105CE0000F931F937B018C0120E030E040E05FE4E4
:105CF000ABD388237CF0C801B70120E030E040E05E
:105D00005FE45ED151D49B01AC0120503040404053
:105D1000504805C0C801B70147D49B01AC01B90187
:105D2000CA011F910F91FF90EF900895A0E0B0E09D
:105D3000EBE9FEE283C7DC012B01FA019C91923072
:105D400008F439C1EB018881823008F433C1943002
:105D500069F4843009F02FC111969C9111978981C3
:105D6000981709F428C1A9EAB2E025C1843009F4E2
:105D700021C18230A9F4923009F01DC19A01AD0110
:105D800088E0EA010990AE01E90109929E01815083
:105D9000C1F7E201898111969C918923818308C111
:105DA000923009F407C112962D903C901397EB01A5
:105DB0008A819B811496AD90BD90CD90DC90179711
:105DC000EC80FD800E811F819101281B390BB901E8
:105DD00037FF04C066277727621B730B603271059B
:105DE0000CF061C0121613066CF537014801062E3F
:105DF00004C096948794779467940A94D2F721E02C
:105E000030E040E050E004C0220F331F441F551F14
:105E10006A95D2F721503040404050402E213F211A
:105E200040235123211531054105510521F021E081
:105E300030E040E050E079018A01E628F72808299F
:105E400019293CC0232BD1F1260E371E35014601FE
:105E5000062E04C096948794779467940A94D2F798
:105E600021E030E040E050E004C0220F331F441F27
:105E7000551F6A95D2F721503040404050402A21AA
:105E80003B214C215D21211531054105510521F0B2
:105E900021E030E040E050E059016A01A628B7282F
:105EA000C828D9280BC0821593052CF01C01AA2400
:105EB000BB24650103C0EE24FF24870111969C9149
:105EC000D20111968C91981709F445C0992339F0A5
:105ED000A80197012A193B094C095D0906C0A601D2
:105EE00095012E193F09400B510B57FD08C0118237
:105EF0003382228224833583468357831DC081E009
:105F000081833382228288279927DC01821B930BAD
:105F1000A40BB50B84839583A683B7830DC0220F92
:105F2000331F441F551F2483358346835783828143
:105F300093810197938382832481358146815781A0
:105F4000DA01C9010197A109B1098F5F9F4FAF4FD6
:105F5000BF4328F30BC0918333822282EA0CFB1CDF
:105F60000C1D1D1DE482F5820683178383E0808368
:105F7000248135814681578157FF1AC0C901AA275C
:105F800097FDA095BA2F81709070A070B070569553
:105F9000479537952795822B932BA42BB52B84837C
:105FA0009583A683B78382819381019693838283AD
:105FB000DF0101C0D201CD01CDB7DEB7E2E15AC6A3
:105FC000A0E2B0E0E5EEFFE245C669837A838B8309
:105FD0009C832D833E834F835887E9E0EE2EF12C7E
:105FE000EC0EFD1ECE010196B701C8D48E010F5EE6
:105FF0001F4FCE010596B801C1D48A8991E0892747
:106000008A8BC701B801AE01475E5F4F8FDEE1D3D7
:10601000A096E6E03BC6A0E2B0E0E0E1F0E31AC6FD
:1060200069837A838B839C832D833E834F83588738
:10603000F9E0EF2EF12CEC0EFD1ECE010196B7011A
:106040009DD48E010F5E1F4FCE010596B80196D4E8
:10605000C701B801AE01475E5F4F68DEBAD3A096B4
:10606000E6E014C6A0E2B0E0E7E3F0E3E7C5698349
:106070007A838B839C832D833E834F835887CE0105
:106080000196BE01675F7F4F79D4CE010596BE01B0
:106090006F5E7F4F73D49985923088F08989823002
:1060A000C8F0943019F4823051F404C0843029F4DB
:1060B000923081F489EA92E0C6C0923049F420E03F
:1060C0009A858A89981321E02A87CE010996BBC058
:1060D000823049F420E09A858A89981321E02A8B3E
:1060E000CE014196B0C02D843E844F8458886D887F
:1060F0007E888F88988CEE24FF248701AA24BB24F5
:10610000650140E050E060E070E0E0E0F0E0C101F7
:1061100081709070892BE9F0E60CF71C081D191DA1
:106120009A01AB012A0D3B1D4C1D5D1D80E090E0E6
:10613000A0E0B0E0E614F7040805190520F481E0BA
:1061400090E0A0E0B0E0BA01A901480F591F6A1F12
:106150007B1FAA0CBB1CCC1CDD1C97FE08C081E079
:1061600090E0A0E0B0E0A82AB92ACA2ADB2A31963A
:10617000E032F10549F0660C771C881C991C569496
:10618000479437942794C3CFFA85EA892B893C89B1
:106190008B859C85280F391F2E5F3F4F17C0CA0182
:1061A00081709070892B61F016950795F794E794AC
:1061B00080E090E0A0E0B0E8E82AF92A0A2B1B2B47
:1061C00076956795579547952F5F3F4F77FDE7CFBA
:1061D0000CC0440F551F661F771F17FD4160EE0C62
:1061E000FF1C001F111F21503040403090E0590724
:1061F00090E0690790E4790760F32B8F3C8FDB0117
:10620000CA018F779070A070B07080349105A1059D
:10621000B10561F447FD0AC0E114F104010511055F
:1062200029F0405C5F4F6F4F7F4F40781A8EFE170A
:1062300011F081E08A8F4D8F5E8F6F8F78A383E09E
:10624000898FCE014996C5D2A096E2E113C5A8E197
:10625000B0E0ECE2F1E3FAC469837A838B839C8338
:106260002D833E834F835887B9E0EB2EF12CEC0E43
:10627000FD1ECE010196B70181D38E010F5E1F4F27
:10628000CE010596B8017AD32985223008F47EC064
:106290003989323010F4B8017CC08A859A898927FF
:1062A0008A87243011F0223031F4231709F06EC0B0
:1062B00069EA72E06EC0343039F41D861E861F868E
:1062C000188A1C861B8604C0323021F484E089873A
:1062D000B7015FC02B853C858B899C89281B390BB6
:1062E0003C872B87ED84FE840F851889AD88BE8896
:1062F000CF88D88CEA14FB040C051D0540F4EE0C85
:10630000FF1C001F111F215030403C872B8720E0CD
:1063100030E040E050E080E090E0A0E0B0E460E0F9
:1063200070E0EA14FB040C051D0540F0282B392B06
:106330004A2B5B2BEA18FB080C091D09B695A7959B
:1063400097958795EE0CFF1C001F111F6F5F7F4F05
:106350006F31710531F7DA01C9018F779070A07044
:10636000B07080349105A105B10561F427FD0AC024
:10637000E114F1040105110529F0205C3F4F4F4F56
:106380005F4F20782D873E874F87588BBE01675F10
:106390007F4FCB011ED26896EAE074C4A8E1B0E05A
:1063A000E3EDF1E357C469837A838B839C832D8368
:1063B0003E834F83588789E0E82EF12CEC0EFD1EBA
:1063C000CE010196B701DAD28E010F5E1F4FCE01CA
:1063D0000596B801D3D28985823038F08989823018
:1063E00020F0C701B80142D301C081E06896E6E021
:1063F0004DC4A8E1B0E0EEEFF1E32CC469837A83E9
:106400008B839C832D833E834F83588789E0E82EBE
:10641000F12CEC0EFD1ECE010196B701AFD28E011C
:106420000F5E1F4FCE010596B801A8D28985823034
:1064300038F08989823020F0C701B80117D301C034
:106440008FEF6896E6E022C4A8E1B0E0E9E2F2E36B
:1064500001C469837A838B839C832D833E834F831E
:10646000588789E0E82EF12CEC0EFD1ECE01019636
:10647000B70184D28E010F5E1F4FCE010596B80181
:106480007DD28985823038F08989823020F0C70139
:10649000B801ECD201C08FEF6896E6E0F7C3A8E13F
:1064A000B0E0E4E5F2E3D6C369837A838B839C830F
:1064B0002D833E834F83588789E0E82EF12CEC0E24
:1064C000FD1ECE010196B70159D28E010F5E1F4FFE
:1064D000CE010596B80152D28985823038F089897B
:1064E000823020F0C701B801C1D201C081E06896B6
:1064F000E6E0CCC3A8E0B0E0EFE7F2E3A8C39B017D
:10650000AC0183E08983DA01C9018827B7FD83954F
:106510009927AA27BB27B82E21153105410551051A
:1065200019F482E0898339C08823A9F0203080E003
:10653000380780E0480780E8580729F460E070E0F9
:1065400080E09FEC2EC0EE24FF248701E21AF30ABC
:10655000040B150B02C079018A018EE1C82ED12CE3
:10656000DC82CB82ED82FE820F831887C801B701DF
:10657000E1D001971816190684F4082E04C0EE0C19
:10658000FF1C001F111F0A94D2F7ED82FE820F83B9
:106590001887C81AD90ADC82CB82BA82CE0101964A
:1065A00018D12896E9E06FC3ACE0B0E0E9EDF2E382
:1065B00055C369837A838B839C83CE010196BE0188
:1065C0006B5F7F4FDBD18D81823061F1823050F182
:1065D000843021F48E81882351F12EC02F8138859B
:1065E00037FD20C06E812F3131051CF06623F9F094
:1065F00023C08EE190E0821B930B29853A854B8561
:106600005C8504C056954795379527958A95D2F7AE
:106610006623B1F050954095309521953F4F4F4FEF
:106620005F4F0EC020E030E040E050E009C02FEFA7
:106630003FEF4FEF5FE704C020E030E040E050E87C
:10664000B901CA012C96E2E025C3A8E0B0E0EAE275
:10665000F3E3FCC27B018C01611571058105910595
:1066600019F482E089835FC083E089838EE1C82EBC
:10667000D12CDC82CB82ED82FE820F831887C80189
:10668000B70158D0FC013197F7FF3BC022273327D1
:106690002E1B3F0B57016801022E04C0D694C794ED
:1066A000B794A7940A94D2F740E050E060E070E01D
:1066B00081E090E0A0E0B0E004C0880F991FAA1F1D
:1066C000BB1F2A95D2F70197A109B1098E219F21FD
:1066D000A023B1230097A105B10521F041E050E0CE
:1066E00060E070E04A295B296C297D294D835E8337
:1066F0006F8378878EE190E08E1B9F0B9C838B834A
:1067000012C0309781F00E2E04C0EE0CFF1C001F4B
:10671000111F0A94D2F7ED82FE820F831887CE1ADA
:10672000DF0ADC82CB821A82CE01019652D02896F3
:10673000EAE0A8C2EF92FF920F931F937B018C01B6
:1067400080E0E81680E0F80681E0080780E018079E
:1067500088F48FEFE816F1040105110531F028F0F7
:1067600088E090E0A0E0B0E017C080E090E0A0E01A
:10677000B0E012C080E0E81680E0F80680E008078C
:1067800081E0180728F088E190E0A0E0B0E004C0C4
:1067900080E190E0A0E0B0E020E230E040E050E0B6
:1067A000281B390B4A0B5B0B04C016950795F79411
:1067B000E7948A95D2F7F701EF54FD4F8081281BAB
:1067C000310941095109C9011F910F91FF90EF90C3
:1067D0000895DF92EF92FF920F931F93FC01E480E4
:1067E000F58006811781D1808081823048F480E075
:1067F00090E0A0E1B0E0E82AF92A0A2B1B2BA5C003
:10680000843009F49FC0823021F4EE24FF248701F4
:1068100005C0E114F1040105110519F4E0E0F0E010
:1068200096C0628173819FEF623879070CF05BC07C
:1068300022E83FEF261B370B2A3131052CF020E0F0
:1068400030E040E050E02AC0B801A701022E04C0A9
:1068500076956795579547950A94D2F781E090E031
:10686000A0E0B0E004C0880F991FAA1FBB1F2A95A3
:10687000D2F70197A109B1098E219F21A023B1234D
:106880000097A105B10521F081E090E0A0E0B0E023
:106890009A01AB01282B392B4A2B5B2BDA01C9015A
:1068A0008F779070A070B07080349105A105B1050C
:1068B00039F427FF09C0205C3F4F4F4F5F4F04C0A2
:1068C000215C3F4F4F4F5F4FE0E0F0E02030A0E011
:1068D0003A07A0E04A07A0E45A0710F0E1E0F0E030
:1068E00079018A0127C06038710564F5FB01E15820
:1068F000FF4FD801C7018F779070A070B0708034BF
:106900009105A105B10539F4E7FE0DC080E490E0E2
:10691000A0E0B0E004C08FE390E0A0E0B0E0E80EBB
:10692000F91E0A1F1B1F17FF05C016950795F79440
:10693000E794319687E016950795F794E7948A9542
:10694000D1F705C0EE24FF248701EFEFF0E06E2FB2
:10695000679566276795902F9F77D794DD24D79406
:106960008E2F8695492F462B582F5D29B701CA01D6
:106970001F910F91FF90EF90DF900895FC01DB01D4
:10698000408151812281622F6F7770E0221F222780
:10699000221F9381892F880F822B282F30E0991F87
:1069A0009927991F11969C93119721153105A9F5E7
:1069B000411551056105710511F482E037C082E887
:1069C0009FEF13969C938E9312979A01AB0167E009
:1069D000220F331F441F551F6A95D1F783E08C9314
:1069E0000DC0220F331F441F551F12968D919C918D
:1069F0001397019713969C938E931297203080E003
:106A0000380780E0480780E4580758F314962D9320
:106A10003D934D935C93179708952F3F310579F47B
:106A2000411551056105710519F484E08C930895B1
:106A300064FF03C081E08C9312C01C9210C02F57DA
:106A4000304013963C932E93129783E08C9387E00B
:106A5000440F551F661F771F8A95D1F770641496EF
:106A60004D935D936D937C93179708951F93DC016D
:106A7000FB019C91923008F447C08081823008F479
:106A800043C0943051F411961C91843099F5818162
:106A9000682F70E0611B71093FC0843021F0923093
:106AA00031F48230B9F18181882389F12DC01196AA
:106AB0001C9111978230F1F081811817D9F4129648
:106AC0002D913C911397828193818217930794F0C3
:106AD00028173907BCF014968D919D910D90BC91AB
:106AE000A02D2481358146815781281739074A070F
:106AF0005B0718F4112341F00AC082179307A4071B
:106B0000B50740F4112319F061E070E005C06FEFA4
:106B10007FEF02C060E070E0CB011F910895629F9B
:106B2000D001739FF001829FE00DF11D649FE00D85
:106B3000F11D929FF00D839FF00D749FF00D659FE6
:106B4000F00D9927729FB00DE11DF91F639FB00DE5
:106B5000E11DF91FBD01CF0111240895991B79E0B2
:106B600004C0991F961708F0961B881F7A95C9F7DD
:106B70008095089597FB092E07260AD077FD04D04B
:106B800049D006D000201AF4709561957F4F089582
:106B9000F6F7909581959F4F0895A1E21A2EAA1BB2
:106BA000BB1BFD010DC0AA1FBB1FEE1FFF1FA217BD
:106BB000B307E407F50720F0A21BB30BE40BF50BBA
:106BC000661F771F881F991F1A9469F76095709543
:106BD000809590959B01AC01BD01CF01089597FB75
:106BE000092E05260ED057FD04D0D7DF0AD0001C91
:106BF00038F450954095309521953F4F4F4F5F4F5A
:106C00000895F6F790958095709561957F4F8F4F19
:106C10009F4F0895AA1BBB1B51E107C0AA1FBB1FB2
:106C2000A617B70710F0A61BB70B881F991F5A9518
:106C3000A9F780959095BC01CD0108952F923F92C0
:106C40004F925F926F927F928F929F92AF92BF927C
:106C5000CF92DF92EF92FF920F931F93CF93DF9328
:106C6000CDB7DEB7CA1BDB0B0FB6F894DEBF0FBE85
:106C7000CDBF09942A88398848885F846E847D84D2
:106C80008C849B84AA84B984C884DF80EE80FD80D4
:106C90000C811B81AA81B981CE0FD11D0FB6F8944A
:106CA000DEBF0FBECDBFED010895EE0FFF1F0590B3
:106CB000F491E02D09944ED080F09F3740F491116B
:106CC0000EF460C060E070E080E89FE3089526F075
:106CD0001B16611D711D811D14C02EC03BD080F09C
:106CE0009F3740F491110EF04DC060E070E080E8F5
:106CF0009FEB089526F41B16611D711D811D01C0B7
:106D00001BC0882371F4772321F09850872B762FAE
:106D100007C0662311F499270DC09051862B70E0AF
:106D200060E02AF09A95660F771F881FDAF7880FC0
:106D30009695879597F908959F3F31F0915020F4EB
:106D4000879577956795B795880F911D9695879547
:106D500097F9089525D0A0F0BEE7B91788F4BB27AE
:106D60009F3860F41616B11D672F782F8827985F1B
:106D7000F7CF869577956795B11D93959639C8F3AA
:106D80000895E894BB2766277727CB0197F90895E4
:106D900057FD9058440F551F59F05F3F71F04795CC
:106DA000880F97FB991F61F09F3F79F087950895B1
:106DB000121613061406551FF2CF4695F1DF08C0D0
:106DC000161617061806991FF1CF869571056105ED
:106DD000089408950F931F93CF93DF93689F8001CA
:106DE000699F100D789F100D1124C8010DD0EC0182
:106DF000009721F060E070E0A8018DD2CE01DF9114
:106E0000CF911F910F910895CF93DF93BC018230F2
:106E1000910510F462E070E0A091AF05B091B0056B
:106E2000ED01E0E0F0E040E050E021C08881998190
:106E30008617970769F48A819B81309719F09383AD
:106E4000828304C09093B0058093AF05FE0134C0E7
:106E50006817790738F44115510519F0841795071B
:106E600008F4AC01FE018A819B819C01E901209715
:106E7000E9F641155105A9F1CA01861B970B049744
:106E800008F4BA01E0E0F0E02AC08D919C911197DE
:106E900084179507F9F46417750781F412968D919C
:106EA0009C911397309719F09383828304C0909339
:106EB000B0058093AF05FD0132964FC0CA01861B15
:106EC000970BFD01E80FF91F6193719302978D9362
:106ED0009C9343C0FD01828193819C01D90110974D
:106EE000A1F68091AD059091AE05892B41F480917A
:106EF000B3039091B4039093AE058093AD05409198
:106F0000B5035091B6034115510541F44DB75EB735
:106F10008091B1039091B203481B590B2091AD05AC
:106F20003091AE0524173507B0F4CA01821B930BCC
:106F30008617970780F0AB014E5F5F4F8417950768
:106F400050F0420F531F5093AE054093AD05F90129
:106F50006193719302C0E0E0F0E0CF01DF91CF9147
:106F60000895CF93DF93009709F450C0EC01229766
:106F70001B821A82A091AF05B091B005109709F15C
:106F800040E050E0AC17BD0708F1BB83AA83FE01C7
:106F900021913191E20FF31FAE17BF0779F48D9164
:106FA0009C911197280F391F2E5F3F4F39832883FB
:106FB00012968D919C9113979B838A83411551055D
:106FC00071F4D093B005C093AF0520C012968D9197
:106FD0009C911397AD01009711F0DC01D3CFFA011A
:106FE000D383C28321913191E20FF31FCE17DF07C4
:106FF00069F488819981280F391F2E5F3F4FFA016C
:10700000318320838A819B8193838283DF91CF9117
:107010000895A0E0B0E0EEE0F8E318CEEC01A8801F
:10702000B980CA80DB80A114B104C104D10441F449
:1070300084E2A82E89EDB82E8BE5C82E87E0D82EE5
:10704000C601B5012DE133EF41E050E0C8DD27EA8C
:1070500031E440E050E063DD7B018C01C601B50105
:107060002DE133EF41E050E0BADDCA01B9012CEE69
:1070700034EF4FEF5FEF53DD6E0D7F1D801F911FCB
:1070800097FF04C0615070408040904868837983C6
:107090008A839B839B01AC015F77B901CA01CDB79D
:1070A000DEB7EAE0EFCDB5CF87EB93E0B2CF6093E8
:1070B000B7037093B8038093B9039093BA0308950C
:1070C000A0E0B0E0E5E6F8E3BFCD8C01009721F445
:1070D000CB019ADE8C01B6C09EEFE92E9FEFF92E10
:1070E000E00EF11E5801A60EB71EAE14BF0408F440
:1070F000A7C08EEF882E8FEF982E8A0C9B1CE7017D
:107100004881598146175707B0F04530510508F4BA
:1071100099C0CA0104978617970708F493C0425094
:107120005040461B570BF401518340837983688399
:10713000C50117DF87C06B01C41AD50AE091AF05FE
:10714000F091B005A0E0B0E0C0E0D0E042C0E815AA
:10715000F905A1F5208131812C153D0578F1C90192
:1071600002968C159D05A8F04E5F5F4F420F531F8E
:10717000E7015983488322813381109729F01396C0
:107180003C932E9312975EC03093B0052093AF05C9
:1071900059C0225030402C193D093183208310976B
:1071A00029F01396FC93EE93129704C0F093B00568
:1071B000E093AF05F7017183608344C080819181C2
:1071C000C817D90708F4EC01DF01828193819C0183
:1071D000F901309709F0BBCF400F511F8091AD05E9
:1071E0009091AE0584179507E9F4C617D707D0F438
:1071F0002091B5033091B6032115310541F42DB727
:107200003EB78091B1039091B203281B390BA216AF
:10721000B306B0F4B092AE05A092AD05E701798354
:10722000688310C0CB01F0DDEC01009749F0F70155
:1072300040815181B80166D0C80193DE8E0102C041
:1072400000E010E0C801CDB7DEB7ECE019CDFC01DD
:1072500088279927E89421912032E9F3293010F00A
:107260002E30C8F32B3239F02D3231F4689403C03C
:1072700027D1820F911D219120532A30C8F31EF48B
:10728000909581959F4F08951F93FC01992788271A
:10729000BC01E89411911032E9F3193010F01E305E
:1072A000C8F31B3249F01D3241F4689405C0F3D095
:1072B000610F711D811D911D119110531A30B8F38A
:1072C0003EF490958095709561957F4F8F4F9F4FBD
:1072D0001F910895911135C1803219F08950855060
:1072E000D0F708959111089581548A5108F4805E71
:1072F000855A08959111089581568A5108F4805253
:1073000085580895FB01DC0102C001900D924150A7
:107310005040D8F70895DC0101C06D9341505040B2
:10732000E0F70895FB01DC010D900020E9F71197CB
:1073300001900D920020E1F70895FC0181918617DC
:1073400021F08823D9F7992708953197CF0108951F
:10735000FB01DC018D91019080190110D9F3990B8B
:107360000895FB01DC0101900D920020E1F70895E2
:10737000FB01DC014150504030F08D9101908019AB
:1073800019F40020B9F7881B990B0895FB01DC0163
:107390004150504048F001900D920020C9F701C0C3
:1073A0001D9241505040E0F70895FC0181E090E0CB
:1073B0000190061609F4CF010020D1F70197089536
:1073C000FB0151915523A9F0BF01DC014D914517F7
:1073D0004111E1F759F4CD010190002049F04D91A0
:1073E00040154111C9F3FB014111EFCF81E090E05D
:1073F00001970895FB019F01E8944230BCF04532AB
:10740000ACF44A3029F497FB1EF4909581959F4F78
:10741000642F7727FFDB805D8A330CF0895D8193D1
:10742000CB010097A9F716F45DE251931082C901D0
:107430008BC0FA01CF93FF93EF9322303CF12532BA
:107440002CF5C22FE894CA3049F497FB3EF490958E
:107450008095709561957F4F8F4F9F4F2C2F3327CD
:1074600044275527FF93EF9398DBEF91FF91605DE1
:107470006A330CF0695D6193B901CA0160507040D4
:107480008040904059F716F4CDE2C19310828F915D
:107490009F91CF9159C0592F482F372F262F660F14
:1074A000771F881F991F660F771F881F991F620F0C
:1074B000731F841F951F660F771F881F991F0895DC
:1074C0007AE0979F902D879F802D910D112408952C
:1074D000FA01CF93FF93EF932230C4F02532B4F436
:1074E000C22F2C2F332744275527FF93EF9355DBCB
:1074F000EF91FF91605D6A330CF0695D6193B901B2
:10750000CA01605070408040904059F710828F91BE
:107510009F91CF9119C0F999FECF92BD81BDF89A84
:10752000992780B50895262FF999FECF1FBA92BDED
:1075300081BD20BD0FB6F894FA9AF99A0FBE019654
:107540000895992788270895DC01FC01672F719120
:107550007723E1F7329704C07C916D937083629139
:0C756000AE17BF07C8F30895F894FFCFE2
:10756C00200043616C426F6F73743A20000200502C
:10757C0049442000203020302030204D0003003BB7
:10758C00003A004D756C7469446973706C617920B4
:10759C00312E312100000001000A000B006400654F
:1075AC00006E006F0004000B0002000600070008CC
:1075BC00000900020020002E0080C094D4FF01FFBF
:1075CC000001FFFE000103FF000103FF00FF0202A8
:1075DC0000FF030100FF0301000101FF00FF03FF97
:1075EC0000FF03FF00FF02FF0002FF0200FF020288
:1075FC00000202FF00FEFFFE000202FF00FF02FF7E
:10760C0000FEFFFE00FF02FF00FEFEFF0001020372
:10761C00000203FE00010203000102030002FEFE51
:10762C000002020200010203000202020001020336
:10763C000001020300FFFEFF00FEFFFE000102FF3F
:10764C0000FE02FF00FF020200FF020200FF020325
:10765C0000FE02FF00FF02FF00FFFEFF00FFFEFF27
:10766C0000FEFFFE00FFFEFE00FEFEFF00FEFFFE22
:10767C0000FEFEFF00FFFEFF00FEFFFE00FFFEFF10
:10768C00000406FF000406050006060600040606B4
:10769C000004060500FE06FE0006060500040605AD
:1076AC0000FE06FE0004060500FEFE0600000000BB
:1076BC0000EE11EE11000000001E1D961C901C53D4
:1076CC001D3A0000000000851DA21D2D00200000A9
:1076DC00000000171F921E00000000D42021213949
:1076EC00217920A4208A20C82000000000EE11215E
:1076FC00213921EE11EE11EE11EE112E00000000D9
:10770C0000EE1121213921000100000000000000D1
:10771C000000010202030303030404040404040430
:10772C0004050505050505050505050505050505FE
:10773C0005060606060606060606060606060606DE
:10774C0006060606060606060606060606060606CD
:10775C0006070707070707070707070707070707AE
:10776C00070707070707070707070707070707079D
:10777C00070707070707070707070707070707078D
:10778C00070707070707070707070707070707077D
:10779C00070808080808080808080808080808085E
:1077AC00080808080808080808080808080808084D
:1077BC00080808080808080808080808080808083D
:1077CC00080808080808080808080808080808082D
:1077DC00080808080808080808080808080808081D
:1077EC00080808080808080808080808080808080D
:1077FC0008080808080808080808080808080808FD
:10780C0008080808080808080808080808080808EC
:0C781C00082000B1050000010000000081
:00000001FF
